:020000040800F2
:1000000028190020F9820008498300084B83000862
:100010004D8300084F830008518300080000000052
:1000200000000000000000000000000053830008F2
:100030005583000800000000578300080F6900087E
:100040005B8300085B8300085B8300085B83000818
:100050005B8300085B8300085B8300085B83000808
:100060005B8300085B8300085B8300085B830008F8
:100070005B8300085B830008656B00085B830008F6
:100080005B8300085B8300085B8300085B830008D8
:100090005B8300085B8300085B8300085B830008C8
:1000A0005B8300085B8300085B8300085B830008B8
:1000B000897100085B8300085B83000815670008EE
:1000C00037630008256700081D6700085B83000888
:1000D0005B8300085B830008D36D00085B83000826
:1000E0005B8300085B8300085B830008DFF80CD0AB
:1000F00008F0D8FB00480047FB160008281900202C
:10010000F0B504460E461546B4FBF5F038B1B4FB25
:10011000F5F72A4631463846FFF7F2FF0646B4FBAC
:10012000F5F005FB1040FDA1085C3070701CF0BDBF
:1001300070B505460C461646022E01DB242E00DD66
:100140000A26002D09DA2D2020703246611C6842F3
:10015000FFF7D6FF0021017006E03246214628460F
:10016000FFF7CEFF00210170204670BD10B5F5A04D
:1001700006F0E3FD10BD2DE9F04105460C462F4683
:100180002646306808F075F980463168424638687E
:1001900008F077F9BDE8F08110B50446EBA006F051
:1001A000CCFD012000F08FFEEFA006F0C6FD0A2076
:1001B00006F0D8FB002006F083FC10BD10B5044605
:1001C000EDA006F0BAFD002000F048FEEDA006F01C
:1001D000B4FD0A2006F0C6FB002006F071FC10BD3D
:1001E00010B50446EBA006F0A8FD2021EF4808F06A
:1001F00015F90020EE490860EE4908702046FFF727
:10020000DDFF10BD2DE9F0410546284608F031F923
:10021000064600F0C6FF0746E6B9E7A006F08DFDEA
:10022000002400BFE94850F8240000B90DE0012087
:10023000A040384204D0E54951F8240006F07DFD85
:10024000202006F066FD641CECE700BFC5A006F0A8
:1002500074FD5BE03246DEA1284608F012F9C8B909
:10026000DDA006F06AFD002400BFD84850F8240045
:1002700000B909E0D54951F8240006F05EFD2020C0
:1002800006F047FD641CF0E700BFB6A006F055FD80
:10029000BDE8F0814FF0000828782D2803D14FF0F9
:1002A00001086D1C761E002400BFC84850F82400C9
:1002B00018B9CFA006F041FD26E0C44850F824103C
:1002C0003246284608F0DDF8E0B9B8F1000F08D052
:1002D000012101FA04F000F05EFFCCA006F02DFD34
:1002E00007E0012101FA04F000F0E0FDCAA006F0E9
:1002F00024FDB64951F8240006F01FFD99A006F030
:100300001CFD01E0641CD0E700BF00BF00BFBFE7D9
:1003100070B505460024C3A006F00FFD00BF1AE02B
:1003200004EB4401C54A52F8210006F006FD0920FD
:1003300006F0EFFC04EB4401C04A02EB810148687F
:1003400006F0FBFC87A006F0F8FC00BF06F0BEFC40
:100350000028FBD0641C0A2CE2D370BDFEB5054614
:10036000284608F086F80646082E20D1002404E02E
:10037000285D08F011F82855641C082CF8D30024D7
:1003800010E0295DAE4808F06BF830B1295D2A19FC
:10039000501C08F065F800B903E0AAA006F0CDFCF7
:1003A000FEBD641C082CECD3284600F09DFCADA0DB
:1003B00006F0C3FC002406E0A148015DAF48005DE3
:1003C0000DF80010641C082CF6D300200DF8040072
:1003D000684606F0B2FC63A006F0AFFC00BFDFE7A2
:1003E00070B50646304608F044F8C5B27DB9A4A001
:1003F00006F0A3FCA1496B394978491EA44A52F87A
:10040000210006F09AFC57A006F097FC70BD2A4622
:100410006FA1304608F035F8C8B99EA006F08DFCF3
:10042000002400BF9A4850F8240000B90AE0984917
:1004300051F8240006F081FC202006F06AFC601CC4
:10044000C4B2EFE700BF47A006F077FCDEE7002468
:1004500000BF8F4850F8240018B993A006F06DFC37
:100460001AE08B4850F824102A46304608F009F864
:1004700078B9601C81496B39487091A006F05DFC29
:10048000834951F8240006F058FC36A006F055FCCC
:1004900002E0601CC4B2DCE700BF00BFB6E77FB576
:1004A00004460D4600262079052815D2DFE800F025
:1004B00003060A0D1100A06806780DE0A06890F907
:1004C000006009E0A068068806E0A068B0F9006056
:1004D00002E0A068066800BF00BF0A2269463046F5
:1004E000FFF726FE684606F028FCADB149A006F0ED
:1004F00024FC0A226946E068FFF71AFE684606F007
:100500001CFC44A006F019FC0A2269462069FFF78A
:100510000FFE684606F011FC7FBD0000303132331B
:100520003435363738394142434445464748494ACD
:100530004B4C4D4E4F505152535455565758595A93
:10054000000000000D0A23200000000052657365C2
:100550007474696E6720746F2064656661756C746D
:10056000732E2E2E0D0A00005265626F6F74696E35
:10057000672E2E2E00000000536176696E672E2EC6
:100580002E0000000D0A5265626F6F74696E672E4F
:100590002E2E00000D0A4C656176696E6720434C73
:1005A00049206D6F64652E2E2E0D0A008C030020ED
:1005B0000000002013020020456E61626C6564201B
:1005C00066656174757265733A2000004C00002006
:1005D0006C69737400000000417661696C61626C43
:1005E000652066656174757265733A2000000000CD
:1005F000496E76616C696420666561747572652008
:100600006E616D652E2E2E0D0A0000004469736127
:10061000626C656420000000456E61626C65642058
:1006200000000000417661696C61626C6520636F57
:100630006D6D616E64733A0D0A0000002891000828
:10064000049700084D75737420626520616E7920EF
:100650006F72646572206F662041455452313233A7
:10066000340D0A0043757272656E7420617373698C
:10067000676E6D656E743A2000000000170400205C
:1006800043757272656E74206D697865723A2000E8
:1006900004000020417661696C61626C65206D69BF
:1006A000786572733A200000496E76616C69642047
:1006B0006D6978657220747970652E2E2E0D0A0092
:1006C0004D697865722073657420746F2000000096
:1006D0000279052A10D2DFE802F0030407080C00B3
:1006E00000BF8368197007E000BF0AB283681A80F0
:1006F00002E08268116000BF00BF70472DE9F0473B
:1007000080464FF000090027404607F0B2FE05463C
:100710002DB1012D28D198F800002A2824D1F5A068
:1007200006F00BFB00241CE004EB8400F74901EB0E
:10073000800604EB8401F54A52F8210006F0FDFA28
:10074000F3A006F0FAFA29463046FFF7A8FEAFF20A
:10075000EC1006F0F2FA00BF06F0B8FA0028FBD061
:10076000641C452CE0D353E0EAA1404607F062FE4A
:100770005FEA00094CD009F101096D1E484607F0F7
:1007800099FE074600243EE004EB8400DF4901EBBC
:10079000800604EB8401DD4A52F8210007F069FE6F
:1007A000824604EB8400D94A52F820105246404653
:1007B00007F067FE30BB04EB8400D44901EB8000F6
:1007C000C068B84219DC04EB840001EB80000069CA
:1007D000B84212DB39463046FFF77AFF04EB84015A
:1007E000CA4A52F8210006F0A8FACBA006F0A5FAF2
:1007F00000213046FFF753FE02E0CAA006F09DFA42
:10080000BDE8F087641C452CBED3D0A006F095FA55
:1008100000BFF5E72DE9FF410746D4A006F08DFAA9
:1008200006F091F84FF47A71B0FBF1F60A226946AE
:100830003046FFF77DFC684606F07FFACFA006F051
:100840007CFA0A226946D2480078FFF771FC6846B4
:1008500006F073FACFA006F070FA0A226946D04873
:100860000078FFF765FC684606F067FACDA006F051
:1008700064FA00F084FC0546CEA006F05EFA00247F
:1008800000BFD14850F8240000B90EE00120A0407C
:10089000284204D0CC4951F8240006F04EFA20201A
:1008A00006F037FA601CC4B2EBE700BF012000F08D
:1008B00051FC48B1C5A006F040FAC649C64A1278B4
:1008C00051F8220006F039FAAFF2683006F035FA36
:1008D000C2A006F032FA0A226946C4480088FFF72F
:1008E00027FC684606F029FAC1A006F026FA05F0B2
:1008F000E4FF06460A226946FFF71AFC684606F03E
:100900001CFAAFF2A03006F018FABDE8FF8110B56E
:100910000446BBA006F011FA10BD2DE9FF41C44802
:10092000007838B90120C2490870C2A006F005FA63
:10093000FFF71CFCCCE106F0D3F90446092C01D0EA
:100940003F2C69D100260027C848D0F80080C84D48
:100950000FE0C648006838B1C44829680268C54835
:1009600007F08FFD00B103E006B92E462F4600BF09
:100970000C35BF4878308542EBD34EB300BFBB493E
:1009800030680968405CB94A39681268895C8842F5
:1009900000D01CE0B54930680968405C48B92021A6
:1009A000B24802680068401CB04B1860B1488154DE
:1009B0000DE0AE4930680968405CAE49AB4A126848
:1009C0008854AA480068401CA8490860D7E700BFBF
:1009D000A648006808B1BE4211D0A7A006F0ADF944
:1009E000354606E0286806F0A8F9092006F091F9D6
:1009F0000C35BD42F6D9FFF7B9FB4FF0000806E011
:100A00009C4911F8080006F084F908F1010897489C
:100A100000688045F4D35AE19448006830B9042C4A
:100A200004D19448FFF7DCFBBDE8FF810C2C05D115
:100A300093A006F082F9FFF799FB48E18B48006824
:100A4000002836D00A2C01D00D2C32D10025AFF26F
:100A5000EC4006F072F900208649844A12688854F6
:100A6000084601900020029088480C230A22804901
:100A7000009001A807F096FC05464DB1286807F0E4
:100A8000F8FC7C490844461C3046A968884702E0C7
:100A90007FA006F052F92021764807F0BFFC002025
:100AA000724908606248007800B9BDE7FFF75EFB55
:100AB0000DE17F2C0ED16D480068C8B100216B4854
:100AC0000068401E694A10606A4A115479A006F015
:100AD00034F9FCE065480068202809D2202C07DBA7
:100AE0007E2C05DC6148006818B9202C01D1EFE0AC
:100AF000EDE0E1E043757272656E742073657474A5
:100B0000696E67733A200D0A00000000A09100088A
:100B1000203D20003D0000002073657420746F208C
:100B2000000000004552523A2056616C7565206104
:100B3000737369676E6D656E74206F7574206F6670
:100B40002072616E67650D0A000000004552523A3E
:100B500020556E6B6E6F776E207661726961626C84
:100B600065206E616D650D0A000000005379737495
:100B7000656D20557074696D653A2000207365635A
:100B80006F6E64732C20566F6C746167653A200039
:100B9000AC010020202A20302E31562028000000F1
:100BA00064010020532062617474657279290D0A12
:100BB0000000000044657465637465642073656EAD
:100BC000736F72733A200000800000204143434855
:100BD000573A200098000020FC0100204379636C04
:100BE000652054696D653A20000000003401002042
:100BF0002C20493243204572726F72733A200000F4
:100C00004166726F333220434C49207665727369B6
:100C10006F6E20322E30204A756C203230203230F8
:100C20003132202F2032333A35323A34340000004A
:100C3000130200200D0A456E746572696E672043C9
:100C40004C49204D6F64652C2074797065202765B0
:100C50007869742720746F2072657475726E2C2009
:100C60006F72202768656C70270D0A000000002055
:100C7000289100088C0300200D1B5B4B0000000036
:100C80001B5B324A1B5B313B314800007701000897
:100C90004552523A20556E6B6E6F776E20636F6DC2
:100CA0006D616E642C20747279202768656C7027E2
:100CB0000000000008200800094801680068401C86
:100CC000074A106007484454204606F022F800BF47
:100CD00005F0EFFF00287FF42EAE00BFA4E6000071
:100CE000000000208C03002070B5064634460CE05E
:100CF0002178FE4807F0B4FB05462DB1A01BC1B218
:100D0000FA482A1AFA488154641C20780028EFD146
:100D100070BD70B5BC22F749F5486B3807F065FB2C
:100D2000002419E0F2486B3890F8291004FB04F015
:100D30001938484300F6C4106043ED496B3991F807
:100D40002810484340F6C41190FBF1F000B2EA4984
:100D500021F81400601CC4B2062CE3DB002454E02C
:100D600004EB8402E24B6B3B93F82A30C3EB420066
:100D70000121002806DDDE4A6B3A92F82A20C2F1F2
:100D80006402D1B2002803DAD94A6B3A92F82A10E9
:100D9000D74A6B3A92F82B2000FB00F35A4301FB31
:100DA00001F392FBF3F2D24B6B3B93F82B30C3F180
:100DB00064031A4442430A2392FBF3F2CC4B6B3B8D
:100DC00093F82A300A2505FB032212B2CB4B23F8F5
:100DD0001420C74A6B3AB2F88620C54B6B3BB3F878
:100DE0008430D21AC54B33F914305A434FF47A7316
:100DF00092FBF3F2BE4B6B3BB3F884301A4412B251
:100E0000BE4B23F81420601CC4B20B2CA8DBB848DE
:100E10006B38B0F89000B6496B39B1F8921088423F
:100E200004DAB3486B38B0F8920012E0B0486B387F
:100E3000B0F89000AE496B39B1F89410884204DDE7
:100E4000AB486B38B0F8940003E0A9486B38B0F8B1
:100E50009000A7496B39A1F8900070BD70B50646A7
:100E600007F0D6F9342007F03DFAA24807F0FEF962
:100E7000042810D100240BE09D4A6B3A11599D4A79
:100E8000A01807F00FFA0546042D00D002E0241D3B
:100E9000BC2CF1D300BF07F0C1F9FFF73AFF26B130
:100EA000012214210F2001F0C3FD70BD90496B3960
:100EB000496801438E4A6B3A5160704700208C4963
:100EC0006B394860704770B505468A48067825B981
:100ED0008B480078864200D170BD894800788449EB
:100EE0006B39087003204870FFF7E8FF0220FFF716
:100EF000DDFF40F6B8307E496B39088128208872C2
:100F00001E20087517208877282179486B38C17210
:100F10001E2141751721C177552101732D2181753E
:100F2000002180F82010102141730F21C175072185
:100F300080F821100B2181730021017680F82210A6
:100F40001421C173082141762D2180F823100E2130
:100F5000017414218176502180F8241046214174B7
:100F60000A21C176142180F82510282181740021DE
:100F7000C174417780F827105A205D496B3981F898
:100F80002800412081F82900002081F82C0081F8F8
:100F90002D0081F82E00322081F82A00002081F8EF
:100FA0002B00002406E0002151481F3820F81410BF
:100FB000601CC4B20E2CF6DB00204D496B39C8878B
:100FC00000214B486B38A0F84010002048496B398D
:100FD0000886002146486B384186818600204449B6
:100FE0006B39888781F84200042081F843004FF470
:100FF000C870A1F846002A20A1F84400414888643E
:101000006E2081F868002B2081F86900212081F88A
:101010006A003DA0FFF768FE002035496B3981F872
:10102000730081F87400142081F87500002081F8A5
:10103000760040F2DC50A1F8780040F24C40A1F874
:101040007A0040F26C70A1F87C00002081F87E00EC
:101050000A2081F87F00C82081F880004FF4966054
:10106000A1F8820040F27E40A1F8840040F23A707C
:10107000A1F886004FF47A70A1F888004FF4C87088
:10108000A1F88A003220A1F88C00012081F88E009E
:1010900040F2DC50A1F890004FF47F70A1F892006C
:1010A0004FF4FA60A1F894000A2081F8960081F8C4
:1010B0009700012081F898004FF47F70A1F89A0002
:1010C0004FF4FA60A1F89C0040F2DC50A1F89E00B9
:1010D0004FF47F70A1F8A0004FF4FA60A1F8A200CD
:1010E00040F2DC50A1F8A40014E0000004970008CE
:1010F0001704002000FC01080C0500201805002042
:10110000B0000020031414004145545231323334EE
:10111000000000004FF41650C1F8A800C820A1F844
:10112000AC00142081F8AE001E2081F8AF00012031
:1011300081F8B0006420A1F8B2004FF49670A1F8D5
:10114000B4004FF4E130C1F8B8000020FFF786FE8C
:1011500000BFC1E6014614480068084201D00120E2
:1011600070470020FCE71049096801430E4A1160EE
:1011700070470D49096881430B4A116070470A485E
:1011800000687047014609484068084201D00120C4
:1011900070470020FCE7054949688143034A5160D4
:1011A0007047024840687047AC000020AC03002044
:1011B00070B5FE48008807F061FA0546FC4907F063
:1011C000DEF9044607F05FFA00B2FA49088070BD04
:1011D0002DE9F04104460D462946204607F0DEFC85
:1011E0000746F54907F0CBF9064607F04CFA00B27E
:1011F000BDE8F0812DE9FE4304460D4694E8070062
:101200008DE807000199686807F0B9F90746009969
:10121000286807F0B4F98046394607F058F90646C1
:10122000A16807F0A9F9A0600199A86807F0A7F9DB
:1012300007460299286807F0A2F98046394607F068
:1012400098F90646216807F042F920600099A868DD
:1012500007F095F907460299686807F090F980460B
:10126000394607F034F90646616807F030F96060E6
:10127000BDE8FE832DE9FF5F002505F04EFB064625
:10128000CE490968701A07F0F9F98046CC4907F091
:1012900076F90746C948066000245FE0C94931F97C
:1012A000140007F0E2F98046394607F068F901A911
:1012B00041F82400C44890F8430000283CDDC249AE
:1012C00091F8430007F0DAF9834659464FF07E5013
:1012D00007F08BF98246BD4931F9140007F0C5F9D2
:1012E0005146009007F04BF98046B74991F843000A
:1012F00007F0C4F9014600904FF07E5007F075F9F1
:1013000083464FF07E5107F037F98246B04850F8D7
:101310002410504607F033F98146414607F0D7F8CC
:10132000AB4941F8240051F8240007F0ACF900B2B1
:10133000A84921F8140005E0A44830F81400A54994
:1013400021F81400A34830F91400A24931F914100F
:1013500000FB01550420FFF7FDFE641C032C9DD308
:101360006420684391490988494390FBF1F501A93C
:101370009948FFF73FFF0420FFF7ECFE18B101A9E1
:101380009648FFF737FF9348B0F90000002803DDC7
:101390009048B0F9000003E08E48B0F900004042E8
:1013A0008449B1F9001088421ADA8A48B0F902007B
:1013B000002803DD8748B0F9020003E08548B0F952
:1013C000020040427B49B1F90010884208DA8148A6
:1013D000B0F90400002803DD01208149487302E0D0
:1013E00000207F494873242D01DDC42D02DB7C4899
:1013F000407B90B300242EE07349B1F8460007F01B
:101400003DF983464FF07E5107F061F88246514620
:101410004FF07E5007F0E9F880466E4931F914002C
:1014200007F023F968490090B1F8460007F026F963
:101430008346694850F82410584607F0A0F88246C1
:10144000009907F044F88146414607F098F8624950
:1014500041F82400641C032CCED30420FFF77AFE4D
:10146000D8B1002417E05F4931F9140007F0FDF806
:1014700081465A4951F824005B4907F080F88246BA
:10148000494607F024F88046584907F078F8534950
:1014900041F82400641C032CE5D34F4A916810687E
:1014A000FFF796FE524908804B4A91685068FFF753
:1014B0008FFE4F494880BDE8FF9F1FB50120FFF711
:1014C00049FE18B102F04CFDFFF7D4FE02F0CFFD4B
:1014D00000240EE03B4830F8140002A921F8140063
:1014E0000120FFF737FE18B90020384921F8140011
:1014F000641C032CEED305F010FA3E49086001F09D
:10150000B9FA05F00AFA3B490968401A40F28A2103
:10151000884206D938480088401C00B23649088005
:1015200009E000BF05F0F9F932490968401A40F2B4
:101530008A218842F6D302F09AFD002427E0214850
:1015400030F8140002A931F81410084400B22DF844
:1015500014003DF91400294931F9141008440321FD
:1015600090FBF1F000B2264921F814003DF9140077
:1015700000EBD0714910214A22F814100120FFF726
:10158000E9FD18B90020114921F81400641C032C4E
:10159000D5D34020FFF7F6FDB0B31A480078A0BBC2
:1015A0000948806C000C174908702FE0FA010020F0
:1015B0007593D83EB40000204C3D0F44E800002055
:1015C00053449231EC000020AC030020F2000020D4
:1015D00080040020F800002068040020740400202B
:1015E000FC040020FE000020000048435E06A33BF0
:1015F000CC000020D800002036010020D0000020C0
:10160000C0000020DE00002027E006E01E48806CBD
:10161000000A48701C48806C887000241AE01B483F
:1016200030F914101A4830F914201A48005D401E91
:1016300002FB0010401C1749095D90FBF1F000B25D
:10164000124921F81400084630F81400104921F816
:101650001400641C032CE2D315E00B4840780128E9
:1016600011D10A48B0F904100B48B0F9000001EBA1
:101670004000032190FBF1F000B204498880084645
:101680008088054908801FBDAC030020C0000020F1
:10169000E2000020DE000020DC00002070B5684879
:1016A000007808B1022000E00020054605F0CFFEDA
:1016B000401BC6B24FF40040624908602C4607E068
:1016C0006148B0F88610204605F0B2FE601CC4B236
:1016D000B442F5DB40F6B83005F044F92C4606E09C
:1016E0004FF47A71204605F0A3FE601CC4B2B442E8
:1016F000F6DB042005F0C1F970BD1CB505F03EF91C
:10170000FFF707FB0020FFF7DEFB4F49D1F8B800D9
:1017100002F0A6FD0120FFF726FD00F0A7F801204A
:10172000FFF730FD8DF801000820FFF72BFD80F05A
:1017300001008DF800004248007808B1012000E067
:1017400000208DF80200404890F89800C0F3C000D7
:101750008DF803003C48B0F88A00ADF804003A4820
:10176000B0F88C00ADF80600684605F0C2FD08B17F
:10177000FFF794FF3548364908604FF4004031497F
:101780000860C01033490861002415E02D4808386E
:10179000006880F400402B49083908602D48C06873
:1017A00080F480502B49C860192005F0DBF819201F
:1017B00005F0D8F8601CC4B20A2CE7DB4FF4805067
:1017C00024490861C0001F49091F086002F078FA27
:1017D000FFF7EEFC0220FFF7D5FC08B102F094FA07
:1017E0000820FFF7CFFC28B104F05BF91A4818492C
:1017F00008600DE00120FFF7C5FC48B14FF4807090
:10180000FFF7C0FC20B11049D1F8A80004F061F83E
:1018100005F083F8114908600B484078052803D18A
:101820004FF4C8700E4908804FF47A700D49088053
:1018300001200D49487301E001F010FCFCE70000B5
:101840001501002014080140AC0300206D2F000892
:101850004C01002000100140D95A0008300100203E
:10186000F6010020F8010020FC04002010B5F94822
:10187000407804280BD0F7484078012807D0F54875
:101880004078052803D0F3484078082802D1012089
:10189000F14908702020FFF775FC10B10120EE49D6
:1018A0000870EC48407812282DD2DFE800F02C15A3
:1018B000191A110920210D1B222627282C2C2C1C3B
:1018C0000020E64908701EE00120E44908701AE093
:1018D0000220E249087016E00320E049087012E097
:1018E00000BF00BF00BF0420DC4908700BE000BF50
:1018F00000BF0620D949087005E000BF00BF0820DE
:10190000D649087000BF00BF10BD10B5D24800789E
:1019100000B910BDCF484078012803D0CD484078A9
:10192000042810D1CE48008981B2002005F080FD46
:10193000C8484078042812D1C948408981B20120A2
:1019400005F076FD0BE0C648008881B2002005F066
:101950006FFDC348408881B2012005F069FD00BFDA
:10196000D7E770B50025BC48007800B102250024F7
:1019700009E0BC4A32F8142091B26219D0B205F0E5
:1019800057FD601CC4B2B54800788442F1DB70BDDD
:1019900070B50546002404E0B24820F81450601CDD
:1019A000C4B2AE4800788442F6DBFFF7DAFF70BDC0
:1019B000F8B5AA48007803284DDDAB48B0F904100B
:1019C000AA48B0F90400002803DDA848B0F90400D3
:1019D00003E0A648B0F9040040426FF06302101A19
:1019E000814210DAA148B0F90400002803DD9F48C5
:1019F000B0F9040003E09D48B0F9040040426FF0E4
:101A00006301081A24E09848B0F904109748B0F927
:101A10000400002803DD9548B0F9040003E0934872
:101A2000B0F904004042643081420EDD8F48B0F9C5
:101A30000400002803DD8D48B0F9040003E08B4862
:101A4000B0F904004042643002E08748B0F9040075
:101A500000B2854988807F48407812287ED2DFE82E
:101A600010F07D00920007014B011200FF05D50127
:101A700063027D009A01F302A303400407057D0081
:101A80007D007D00C4057948C188774800880844F6
:101A900000B2744908807548C08873490988494272
:101AA000084400B26F4948806A4890F98E006E4938
:101AB000B1F90410484300F2DC506B49B1F902104F
:101AC0000844B0F57F7F02DA4FF47F701FE0614871
:101AD00090F98E006449B1F90410484300F2DC50DB
:101AE0006149B1F902100844B0F5FA6F02DD4FF414
:101AF000FA600CE0574890F98E005B49B1F9041088
:101B0000484300F2DC505849B1F90210084400B2D1
:101B1000534908814F4890F98E005349B1F9041098
:101B2000484300F2DC505049B1F90210401AB0F5B8
:101B30007F7F02DA4FF47F7021E0464890F98E00F3
:101B40004949B1F90410484300F2DC504649B1F963
:101B50000210401AB0F5FA6F04DD00E073E24FF4B2
:101B6000FA600CE03B4890F98E003F49B1F904104F
:101B7000484300F2DC503C49B1F90210401A00B26F
:101B8000374948815FE23848B0F9020080000321FC
:101B900090FBF1F03549C988084400B2314908800A
:101BA0003148B0F9020040004042032190FBF1F1BE
:101BB0002E48C0882C4A128852421044084400B271
:101BC000284948802848B0F90200400040420321DB
:101BD00090FBF1F12548C28823480088104408444E
:101BE00000B2204988801B48B0F89000194991F94B
:101BF0008E101D4AB2F9042001FB02001549B1F80C
:101C00009210884203DA1348B0F892001EE011489F
:101C1000B0F890000F4991F98E10134AB2F90420E0
:101C200001FB02000B49B1F89410884203DD09481A
:101C3000B0F894000AE00748B0F89000054991F91F
:101C40008E10094AB2F9042001FB020000B20449D7
:101C5000088197E7AC030020150100201401002043
:101C6000160100208C040020C2010020B0010020D9
:101C7000FE48C0880146FE4840880144FD4890F96E
:101C80008E00FB4A928850434042084400B2FA4911
:101C90000880F648C088F649098849420844014648
:101CA000F44890F98E00F24A928800FB021000B2CC
:101CB000F1494880ED48C188ED4800880844014654
:101CC000EC4890F98E00EA4A928800FB021000B2BC
:101CD000E9498880E548C088E54949884942014486
:101CE000E44890F98E00E24A92885043404208440A
:101CF00000B2E149C88045E7DC48C088DC49098872
:101D000049420144DA4840880144DA4890F98E009B
:101D1000D74A928850434042084400B2D6490880CE
:101D2000D248C088D249098849420844D0494988E4
:101D300049420144CF4890F98E00CD4A928800FB79
:101D4000021000B2CC494880C848C188C848008801
:101D50000144C74840880144C64890F98E00C44AEF
:101D6000928800FB021000B2C3498880BF48C18836
:101D7000BF4800880844BE49498849420144BD48DB
:101D800090F98E00BA4A928850434042084400B20B
:101D9000B949C880F6E6B548C0880146B4484088CD
:101DA0000144B44890F98E00B14A928850434042B1
:101DB000084400B2B0490880AC48C088AC490988E2
:101DC00049420844AA4949884942084400B2AA49FC
:101DD0004880A648C0880146A54840880144A548D7
:101DE00090F98E00A24A928800FB021000B2A2492C
:101DF00088809E48C1889E48008808449C4949883C
:101E00004942084400B29C49C880BBE69848B0F9F2
:101E100002008000032190FBF1F09449C98801443D
:101E2000944890F98E00924A928800FB021000B20A
:101E3000914908808E48B0F90200400040420321D9
:101E400090FBF1F08949C988894A128852421144AD
:101E50000144884890F98E00854A92885043404258
:101E6000084400B2844948808148B0F9020040002B
:101E70004042032190FBF1F27C48C1887C480088F5
:101E8000084411187B4890F98E00794A9288504393
:101E90004042084400B2784988807548B0F9020091
:101EA0008000032190FBF1F07049C988014471481A
:101EB00090F98E006E4A928850434042084400B226
:101EC0006D49C8806A48B0F90200400040420321D1
:101ED00090FBF1F06549C988654A12885242114465
:101EE0000144644890F98E00614A928800FB021018
:101EF00000B2614908815E48B0F9020040004042EA
:101F0000032190FBF1F15948C288594800881044D8
:101F10000144584890F98E00554A928800FB0210FF
:101F200000B2554948818EE0514AB2F90020514231
:101F300001EBD1724D4BDB8803EB62034C4AB2F9E3
:101F4000020000EBD07203EB62034A4A92F98E2042
:101F5000474EB68802FB063212B2474B1A80444AFB
:101F6000B2F90020514201EBD172404BDB8803EB08
:101F700062023F4BB3F90230584200EBD07302EBE0
:101F800063033C4A92F98E20394EB688724352421E
:101F90001A4412B2384B5A80354AB2F9001001EB9C
:101FA000D172324BDB8803EB6203314AB2F9020093
:101FB00000EBD07203EB62032E4A92F98E202C4E76
:101FC000B68802FB063212B22B4B9A80284AB2F92D
:101FD000001001EBD172254BDB8803EB6202244B2E
:101FE000B3F90230584200EBD07302EB6303214A8D
:101FF00092F98E201E4EB688724352421A4412B293
:102000001D4BDA801948C088194949884942014462
:10201000184890F98E00164A928800FB021000B210
:10202000194608811148C08801461148408801447A
:10203000104890F98E000E4A92885043404208445E
:1020400000B219464881AEE30948B0F900008000AB
:102050004042052190FBF1F00449C9880844044935
:10206000B1F9021001EBC1010A2207E0B001002022
:10207000C2010020AC0300208C04002091FBF2F18F
:102080000144F74890F98E00F64A928800FB02104E
:1020900000B2F5490880F348B0F9000080004042E2
:1020A000052190FBF1F0F149C9880844ED49B1F9E7
:1020B0000210494201EBC1010A2291FBF2F10144F5
:1020C000E74890F98E00E74A928800FB021000B2C0
:1020D000E5494880E348B0F900008000052190FB05
:1020E000F1F0E249C9880844DE49B1F9021001EB78
:1020F000C1010A2291FBF2F10144D94890F98E0006
:10210000D84A928850434042084400B2D649888059
:10211000D448B0F900008000052190FBF1F0D349CC
:10212000C9880844CF49B1F90210494201EBC10105
:102130000A2291FBF2F10144C94890F98E00C94A84
:10214000928850434042084400B2C749C880C548FD
:10215000B0F9000080004042052190FBF1F0C34936
:10216000C98808440146BE4890F98E00BD4A92884D
:1021700050434042084400B2BB490881B948B0F915
:1021800000008000052190FBF1F0B849C98808449F
:102190000146B34890F98E00B24A928800FB0210C3
:1021A00000B2B1494881FEE2B048C088AD49098813
:1021B00049420144AB4840880144A94890F98E0047
:1021C000A84A928850434042084400B2A649088079
:1021D000A648C088A349098849420844A1494988BA
:1021E000494201449E4890F98E009E4A928800FB25
:1021F000021000B29C4948809C48C18899480088D8
:102200000144984840880144954890F98E00954AC9
:10221000928800FB021000B2934988809348C188DD
:102220009048008808448F494988494201448C48B5
:1022300090F98E008B4A928850434042084400B285
:102240008949C8808948C08886490988494201442B
:10225000844840880144824890F98E00814A9288DF
:1022600000FB021000B2804908818048C0887D4987
:102270000988494208447B494988494201447848D1
:1022800090F98E00774A928850434042084400B249
:10229000754948817548C188724800880144714871
:1022A000408801446E4890F98E006E4A92885043EF
:1022B0004042084400B26C4988816C48C188694832
:1022C000008808446749498849420144644890F9B4
:1022D0008E00644A928800FB021000B26249C881F5
:1022E00061E26048B0F90000C0EBC0000A2190FB39
:1022F000F1F05E49C98808445A49B1F90210A1EBCE
:10230000C1010A2291FBF2F10144554890F98E0077
:10231000544A928800FB021000B253490880514889
:10232000B0F90000A0EBC0000A2190FBF1F04F498A
:10233000C98808444B49B1F90210A1EBC1010A2236
:1023400091FBF2F10144464890F98E00454A92888B
:1023500000FB021000B2444948804248B0F9000036
:10236000A0EBC0000A2190FBF1F04049C988084465
:102370003C49B1F90210C1EBC1010A2291FBF2F113
:102380000144374890F98E00364A928800FB0210CB
:1023900000B2354988803348B0F90000C0EBC00076
:1023A0000A2190FBF1F03149C98808442D49B1F95F
:1023B0000210C1EBC1010A2291FBF2F1014428484D
:1023C00090F98E00274A928800FB021000B226493D
:1023D000C8802648C088234949884942014420488A
:1023E00090F98E001F4A928850434042084400B240
:1023F0001D4908811D48C0881A4909884942084476
:102400000146174890F98E00164A92885043404280
:10241000084400B2144948811448C0880146114854
:10242000408801440E4890F98E000E4A928850432D
:102430004042084400B20C4988810C48C1880948D0
:10244000008808440146064890F98E00054A9288A3
:1024500050434042084400B20349C881A3E1000050
:10246000AC030020C20100208C040020B001002039
:10247000FE49CA88FE4909881144FD4AB2F9022082
:10248000504200EBD07201EB6202FA4991F98E10D2
:10249000F74B9B8801FB032109B2F74A1180F449ED
:1024A000B1F90010484200EBD071F04AD28802EB3B
:1024B0006101EF4A528852420A44EE4991F98E1066
:1024C000EB4B9B8801FB032109B2EB4A5180E749A2
:1024D000C988E74A128852420A44E549B1F9020024
:1024E00000EBD07102EB6102E24991F98E10E04BF2
:1024F0009B8801FB032109B2DF4A9180DC49B1F9D5
:10250000000000EBD071D94AD28802EB6102D849B1
:1025100049880A44D74991F98E10D54B9B8801FB15
:10252000032109B2D44AD180D149B1F9000000EBAE
:10253000D071CE4AD28802EB6101CD4A5288524214
:102540000A44CC4991F98E10C94B9B8859434942A2
:10255000114409B2C84A1181C449C988C44A1288C1
:1025600052421144C24AB2F90220504200EBD072EA
:1025700001EB6202BF4991F98E10BD4B9B88594314
:102580004942114409B2BC4A5181B949B1F900101C
:10259000484200EBD071B54AD28802EB6102B449DF
:1025A00049880A44B34991F98E10B14B9B8859432D
:1025B0004942114409B2B04A9181AC49CA88AC4938
:1025C00009880A44AA49B1F9020000EBD07102EB74
:1025D0006102A84991F98E10A54B9B885943494245
:1025E000114409B2A44AD181DDE0A048C088014667
:1025F0009F48408801449F4890F98E009C4A9288E9
:1026000000FB021000B29C4908809848C088984995
:10261000098849420844964949884942084400B219
:10262000954948809148C0880146914840880144B6
:10263000904890F98E008E4A928850434042084458
:1026400000B28D4988808948C1888948008808443B
:10265000874949884942084400B28749C880A2E0B6
:10266000844B93F99630854EB6F9026003FB06F26F
:10267000D31702EB13737F4EB6F89E6006EB23135D
:102680007A4EB6F9026033447A4EB6F89A60B34295
:1026900003DA784BB3F89A3030E0764B93F9963002
:1026A000764EB6F9026003FB06F1CB1701EB13730C
:1026B000704EB6F89E6006EB23136C4EB6F90260BE
:1026C00033446C4EB6F89C60B34203DD694BB3F8FB
:1026D0009C3013E0674B93F99630684EB6F9026070
:1026E00003FB06F0C31700EB1373624EB6F89E604F
:1026F00006EB23135D4EB6F9026033441BB2604E05
:1027000033805C4B93F997305C4EB6F9006003FB65
:1027100006F2D31702EB1373564EB6F8A46006EB1D
:102720002313524EB6F900603344524EB6F8A060FF
:10273000B34203DA4F4BB3F8A03030E04D4B93F97E
:1027400097304E4EB6F9006003FB06F1CB1701EB54
:102750001373484EB6F8A46006EB2313434EB6F944
:1027600000603344434EB6F8A260B34203DD414BF0
:10277000B3F8A23013E03F4B93F997303F4EB6F9D0
:10278000006003FB06F0C31700EB1373394EB6F875
:10279000A46006EB2313354EB6F9006033441BB238
:1027A000374E738000BF00BF2020FEF7EBFC0028EF
:1027B0006DD0002000902F4890F8980010F0010F85
:1027C00005D12C4890F8980010F0020F08D02D4841
:1027D00080892849B1F87810401A80B2ADF800001D
:1027E000244890F8980010F0040F08D12548C089BB
:1027F0002049B1F87810401A80B2ADF802001D48A7
:10280000B0F89E00BDF80010084400B21C490880D2
:102810001848B0F8A400BDF80210084400B21849E6
:1028200048801948C07888B3124991F99610134A24
:10283000B2F9022001FB02F0C11700EB1171104A3E
:10284000128802EB211109B20D4A1180094991F950
:1028500097100A4AB2F9002001FB02F0C11700EB01
:102860001171074A528802EB211111E0B0010020DA
:10287000C2010020AC0300208C040020CC0000200A
:10288000160100203C0100202E05002003E03FE05F
:1028900009B2614A51806048B0F900005F49B1F85F
:1028A0009A10884203DA5D48B0F89A000EE05A4860
:1028B000B0F900005949B1F89C10884203DD57482F
:1028C000B0F89C0002E05448B0F9000000B2524950
:1028D00008800846B0F902005049B1F8A0108842BB
:1028E00003DA4E48B0F8A0000EE04B48B0F9020001
:1028F0004A49B1F8A210884203DD4848B0F8A20066
:1029000002E04548B0F9020000B24349488000BFE8
:10291000424890F8980010F0080F0DD0002409E00C
:10292000221D3F4B33F8122091B2A21DD0B204F009
:102930007FFD641C042CF3D33A48B0F90050012405
:1029400008E0384830F91400A84202DD354830F973
:102950001450641C344800788442F2D3002455E0BB
:102960002E48B0F88600A8420BDA2E4830F8140042
:102970002A49B1F88610691A401A00B2294921F88B
:102980001400284830F914002449B1F88410884212
:1029900003DA2248B0F884000EE0224830F914002F
:1029A0001E49B1F88610884203DD1C48B0F8860045
:1029B00002E01C4830F9140000B21A4921F8140052
:1029C0001748B0F906001549B1F87A10884212DAB2
:1029D0001020FEF7D7FB38B91048B0F8840000B2D9
:1029E000104921F8140006E00C48B0F8880000B245
:1029F0000C4921F814000D48407830B90748B0F868
:102A0000880000B2074921F81400641C06480078C9
:102A10008442A5D3F8BD000016010020AC030020BD
:102A20003C0100208C04002014010020FC04002044
:102A30002DE9F04104460D4616464FF0000815E01A
:102A400000270AE0FA48C06880F48050F849C8605E
:102A5000284603F087FF781CC7B2A742F2DB3C2070
:102A600003F080FF08F1010000F0FF08B045E7DB4C
:102A7000BDE8F0812DE9F04F87B04FF00008ED4838
:102A8000B0F9060040F2DC51884201DA64271CE00C
:102A9000E848B0F90600B0F5FA6F10DAE64890F8A9
:102AA0002E00E449B1F90610A1F2DC5148434FF47D
:102AB000FA7190FBF1F0C0F16400C7B205E0DE48A6
:102AC00090F82E00C0F16400C7B20024BFE0D948DE
:102AD00030F91400D849B1F87810401A002807DD01
:102AE000D44830F91400D449B1F87810401A06E0FF
:102AF000D148B0F87800CF4931F91410401AB0F538
:102B0000FA7F18DACB4830F91400CB49B1F87810C5
:102B1000401A002807DDC74830F91400C649B1F84B
:102B20007810401A09E0C448B0F87800C14931F97A
:102B30001410401A01E04FF4FA7085B2022C40D014
:102B4000BD4890F8730058B1BB4890F87300A84294
:102B500005DAB94890F87300281A85B200E000251C
:102B6000642095FBF0F086B2B449701C31F9100076
:102B700031F91610401A06EBC60101EB0611A5EB60
:102B800081014843642190FBF1F0AC4931F8161003
:102B9000084400B2AA4921F81400A74890F82C0074
:102BA00068434FF4FA7190FBF1F0C0F1640000F05B
:102BB000FF0A0AFB07F0642190FBF1F000F0FF0A26
:102BC0001FE09D4890F8740058B19B4890F874003D
:102BD000A84205DA984890F87400281A85B200E0F7
:102BE000002528B2964921F81400934890F82D004A
:102BF00068434FF4FA7190FBF1F0C0F1640000F00B
:102C0000FF0A8D480A30005D00FB0AF0642190FB4A
:102C1000F1F08C49085588481E30005D00FB0AF031
:102C2000642190FBF1F088490855824830F914007E
:102C30008149B1F87810884207DA814830F81400E9
:102C4000404200B27E4921F81400601CC4B2032C3B
:102C5000FFF63DAF7748B0F906007749B1F87A1032
:102C6000884203DA7448B0F87A000BE07148B0F992
:102C70000600B0F5FA6F02DD4FF4FA6002E06D482D
:102C8000B0F9060085B26C48B0F87A00281A4FF403
:102C90007A7148436849B1F87A10C1F5FA61B0FB1E
:102CA000F1F085B2642095FBF0F086B26749701CA4
:102CB00031F9100031F91610401A06EBC60101EB8C
:102CC0000611A5EB81014843642190FBF1F05F49B7
:102CD00031F81610084400B25949C8805C48407A5F
:102CE000002855D05B49B1F900105B4AB2F90020C9
:102CF000881A05F0BAFC5949029005F040FC834659
:102D0000574905F072FC0690069806F071F8059098
:102D1000069806F02DF904904949B1F9000005F034
:102D2000A4FC0090049905F02AFC83464449B1F9BB
:102D3000020005F09AFC0090059905F020FC594628
:102D4000019005F0C4FB029005F09DFC00B20390D9
:102D50003B49B1F9020005F088FC0090049905F0A8
:102D60000EFC37490290B1F9000005F07EFC00909E
:102D7000059905F004FC0190029905F0FAFB8346E1
:102D800005F081FC00B22E4908800398488000BFFE
:102D90000220FEF7F7F9E8B332480078401CC0B2D1
:102DA00030490870062190FBF1F201FB120060BB74
:102DB00004F010F92C4991F800B00978491C2A4A0E
:102DC00011704FEAEB710BEB5171C910ABEBC10104
:102DD000264A22F811004FF0000909E0234830F894
:102DE000190040441FFA80F809F1010000F0FF09C2
:102DF000B9F1080FF2DBC3464FEAE87108EB5171F5
:102E0000C81000F063FF1A49087019480078194982
:102E1000098800E035E0884206DC074890F86A003F
:102E200013490978884229DD00201349087028E0F9
:102E3000001001403C010020AC0300200C050020E4
:102E4000B0010020B8010020BE01002018050020BC
:102E5000FC0400200E020020AA010020DB0F4940E4
:102E6000000034436D0100206E0100209C0400200E
:102E7000AC010020F40100206C0100200420FE4978
:102E80000870FD48007802F00DFFFC48008800281B
:102E900003DD0120FEF75EF918B9F9480088002823
:102EA00006DDF848C06880F48050F649C8601BE031
:102EB000F548C07818B14FF48050F2490861F248E3
:102EC000407818B14FF48050EE4948614FF40060EB
:102ED000FEF758F940B1EC49497809B1012100E009
:102EE0000021084603F0BEF8E8480068E849096890
:102EF000884215D9E448407B78B90020E249C8707F
:102F0000E048C06880F48050DE49C860DF4800684F
:102F1000E0490844DE49086002E00120DA49C8704F
:102F200001F09EFC1020FEF715F9A8B1D748006803
:102F3000D949096888420FD9D848007805280BDBA1
:102F4000D2480068D6490844D3490860D54800688B
:102F500080F40040D3490860D348C06818B1D24813
:102F6000C168D248884707B0BDE8F08F70B5054604
:102F7000CF49485D04F065FA044640F2EE208442F1
:102F800003DB40F6CA00844203DDC9486B38B0F861
:102F90007840204670BD70B5C6480078401CC549D1
:102FA0000870002457E02046C3490968884700B2EA
:102FB000C0490E78F11706EB91718910A6EB8101DB
:102FC000BE4A02EBC40222F811000020BC4921F8DD
:102FD000140000250EE0B94800EBC40030F81500DD
:102FE000B74931F81410084400B2B54921F814006B
:102FF000681CC5B2042DEEDBB14931F91410881CF0
:10300000C11700EB91718910AD4A22F814101046D7
:1030100030F91410AB4830F91400C01E814207DAB1
:10302000104630F81400801C00B2A64921F81400A4
:10303000A34830F91410A34830F91400C01C814291
:1030400007DD9F4830F81400801E00B29D4921F82A
:103050001400601CC4B2082CA5DB70BD2DE9F04F34
:1030600089B00020079002F034FD08B1FFF793FF0C
:10307000864800689449096888427DD98348006879
:1030800044F620610844904908600820FEF77AF869
:1030900008B9FFF780FF4FF40070FEF773F80028BF
:1030A00054D083486B3890F87F0000EB800087494C
:1030B000B1F90010884231DA7348407870B30025C6
:1030C00009E07B486B38B0F8780000B27D4921F800
:1030D0001500681CC5B2032DF3DB75486B38B0F8DA
:1030E000820000B27749C88071486B3890F87F0041
:1030F0006F496B3991F88010084400EB80007349E8
:10310000B1F90010884203DA00205F494870087066
:103110006F480088401C00B26D49088064486B38D5
:1031200090F87F0000EB80006849B1F900108842F8
:1031300006DA5548407818B900205349487008709D
:1031400062480088401C00B2604908805D48B0F9C0
:10315000060057496B39B1F87A1088426ADA0020C4
:103160005C490880488088805B49088048805B48CB
:103170000078401C594900E0E5E208705148B0F978
:1031800004004B496B39B1F87A1088421CDA4D487B
:10319000B0F9020046496B39B1F87A10884213DA67
:1031A0003948407880B94D48007814280BD14FF445
:1031B0007A70334908804FF48070FDF7E3FF0028F0
:1031C00001D002F09EFB93E10420FDF7DBFF80B30A
:1031D0002D48407868BB3B48B0F9040034496B394E
:1031E000B1F87A10884234DA3648B0F90200304932
:1031F0006B39B1F87C1088422BDD3248B0F9000001
:103200002B496B39B1F87C10884222DD33480078B5
:103210001428D8D13248008830B1002030490880C5
:1032200001203049088063E12F48008818B9012047
:1032300002E00EE0C6E000202B4908800846008826
:1032400018B102202949087052E10320274908706B
:103250004EE117486B38B0F8560000285BDD244873
:10326000407938B10848007820B1012006494870FB
:10327000204841E045E000006C010020F6010020FC
:10328000F801002000100140FC0400202C01002067
:103290006801002020A1070070010020E00100204B
:1032A000F04902000C08014070050020AE0100202A
:1032B00017040020740100204C010020AC04002001
:1032C000EC0400203C010020940100203801002083
:1032D0003A010020880100208E01002075010020A5
:1032E0005E01002060010020F20100202801002082
:1032F0002E0500200E020020B0F90000F9490880D8
:1033000005E0F948407810B10020F74948700020E6
:10331000F6490870ECE0F648B0F90400F549B1F858
:103320007A1088420CDBF34890F87E00012812D115
:10333000EF48B0F90000EF49B1F87A1088420ADA94
:10334000E948407838B1E94800781428E2D10020F3
:10335000E5494870CCE0E648B0F90400E549B1F829
:103360007C1088420CDCE248B0F90000E149B1F879
:103370007C10884222DDDF4890F87E0001281DD1B4
:10338000DB48B0F90200DB49B1F87C10884215DA5D
:10339000D548407890B9D848008878B9D248C078E4
:1033A00060B1D2480078142807D10120CE49487076
:1033B000D248B0F90000CB49088099E00020CB4901
:1033C000087095E0CA48B0F90600CA49B1F87C1007
:1033D000884220DDC448407800281CD1C448B0F998
:1033E0000400C449B1F87A10884215DAC048B0F92F
:1033F0000200C049B1F87A1088420DDABB48007863
:10340000142803D14FF4C870BD490880B74800782C
:10341000401CB64908706BE0B548B0F90400B549E6
:10342000B1F87C10884214DDB148B0F90200B1490E
:10343000B1F87A1088420CDAAC480078142802D12E
:103440000120A9498873A9480078401CA749087041
:103450004EE0A748B0F90200A649B1F87C108842B6
:103460000BDDA448B0F84000801C01B2A148A0F8D0
:1034700040100120FDF7F2FC3AE09D48B0F902004F
:103480009C49B1F87A1088420BDA9A48B0F84000AB
:10349000801E01B29748A0F840100120FDF7DEFC25
:1034A00026E09348B0F900009249B1F87C108842B8
:1034B00009DD9048C08F801C00B28E49C88701206A
:1034C000FDF7CCFC14E08A48B0F900008949B1F856
:1034D0007A10884209DA8748C08F801E00B2854979
:1034E000C8870120FDF7BAFC02E000207F49087080
:1034F0000420FDF747FE10B38248008898B17A484F
:10350000407880B17A48B0F906007A49B1F87A106B
:10351000884208DD7C48407928B932207B49088000
:103520000020784908807848007A48B178480088B7
:1035300028B97848008810B93220744908800BE017
:103540007448008840B16848407828B90020714923
:10355000088001207049088000253BE0281D64494F
:1035600031F9100040F21451884201DA012000E0E4
:10357000002005EB45018840291D5D4A32F91110F4
:1035800040F21452914209DD291D594A32F91110B5
:1035900040F2A462914201DA012100E0002105EB32
:1035A0004502521C91400843291D514A32F911101D
:1035B00040F2A462914201DD012100E0002105EB0F
:1035C0004502921C914008430799084380B2079036
:1035D000681CC5B2042DC1DB00250EE045484C3007
:1035E00030F8150007990840002801DD012000E0AF
:1035F000002045494855681CC5B20E2DEEDB4248F7
:10360000007848B93B4890F87F0000EB80004349C0
:10361000B1F9001088420EDA0120FDF79BFD50B190
:103620003148007950B900203D4908804880012088
:103630002D49087102E000202B4908713248407979
:1036400010B90120284908702748007920B14FF4AB
:1036500000403449086004E04FF400403149091F3C
:1036600008601020FDF776FD88B31F48C07A70B35C
:103670002D48007805282EDB2348807968B11A4848
:10368000C07968B901201849C8712849081F02F09B
:1036900074F902202649087002E000201249C8711E
:1036A0001948C079A0B11048007A80B901200E49AC
:1036B000087220480068204908601E484068486039
:1036C000091D081F02F059F901201949087002E08C
:1036D0000020054908720C48007A78B3012002499D
:1036E00088724FE0AA010020FC0400207501002030
:1036F0003C010020AC030020F80100200E02002055
:10370000F6010020F20100202E0500205C010020BF
:10371000620100205E0100206001002038010020CD
:103720008E01002014080140E0010020D401002097
:103730005A010020C8010020D8010020FFE7002026
:10374000FE4988721EE0FE4991F900000978491C83
:1037500049B2FB4A1170C11700EB91718910B0EBAF
:10376000810106D0012905D0022904D0032904D102
:1037700002E006E005E004E003E00020F049087004
:1037800000BF00BF03F0C9F8EE49086008460068B2
:10379000ED49096888427DD9EC480089E949096802
:1037A0000844E9490860FDF788FE03F0B6F8E549EA
:1037B000086008460068E6490968401AE54908803B
:1037C000E0480068E24908601020FDF7C3FC0028CB
:1037D0000AD0DA48C07910B9D848007A10B1D74871
:1037E000007B10B902F0A6F810E1DB48B0F9000048
:1037F00004F03BFFD949039004F0C1FE049005F0AA
:10380000B7FB0690D448B0F9000004F02EFFD3496E
:10381000039004F0B4FE049005F0EAFA0590CB485A
:1038200090F8AF00B8B3CE49B1F90210CD4AB2F961
:103830000220881A01F010F9C44991F8AF104942EA
:10384000884204DAC14890F8AF0040421AE0C44907
:10385000B1F90210C34AB2F90220881A01F0FCF84B
:10386000BA4991F8AF10884203DDB84890F8AF002C
:1038700008E0BB49B1F90210BA4AB2F90220881A2D
:1038800001F0EAF8B7494988084401B2B5484180D7
:10389000B34901E0FDE176E0B1F900100246B2F96A
:1038A0000020881A01F0D8F8A84991F8AF104942D1
:1038B000884204DAA54890F8AF0040421AE0A849CF
:1038C000B1F90010A74AB2F90020881A01F0C4F833
:1038D0009E4991F8AF10884203DD9C4890F8AF00F4
:1038E00008E09F49B1F900109E4AB2F90020881AF9
:1038F00001F0B2F89B490988084401B29948018057
:103900000146B1F9000004F0B0FE0090069904F001
:1039100036FE94490290B1F9020004F0A6FE009030
:10392000059904F02CFE0190029904F022FE8E49C4
:10393000039004F05AFE049004F0A5FE00B28B49F7
:1039400008808849B1F9000004F08FFE00900599C5
:1039500004F015FE83490290B1F9020004F085FEDF
:103960000090069904F00BFE0190029904F0AFFD5F
:103970007D49039004F039FE049004F084FE00B207
:103980007A49488041E07649B1F9000004F06DFEC3
:103990000090069904F0F3FD71490290B1F902001C
:1039A00004F063FE0090059904F0E9FD019002998E
:1039B00004F0DFFD6C49039004F017FE049004F05E
:1039C00062FE00B2694908806549B1F9000004F05F
:1039D0004CFE0090059904F0D2FD61490290B1F9C6
:1039E000020004F042FE0090069904F0C8FD019028
:1039F000029904F06CFD5C49039004F0F6FD04901C
:103A000004F041FE01B25948418000BF002437E173
:103A10004A480079F0B3022C77DA554830F914009F
:103A2000524931F91410C1EB400010F5FA7F01DA68
:103A3000504815E04E4830F914004C4931F9141043
:103A4000C1EB4000B0F5FA7F02DD4FF4FA7007E0F9
:103A5000474830F91400454931F91410C1EB4000D2
:103A6000454931F81410411A38483E3030F81400F6
:103A7000084406B23548407C7043642190FBF1F065
:103A800007B2324890F82500404200EB8000B8426F
:103A900008DD00E039E02D4890F82500404200EBB9
:103AA00080000DE0294890F8250000EB8000B84226
:103AB00005DA264890F8250000EB800000E0384643
:103AC00007462E4830F9140030442D49884201DA67
:103AD00008460DE0294830F91400304442F21071D4
:103AE000884201DD084603E0244830F914003044E0
:103AF00000B2224921F81400084630F91400134995
:103B0000C97E48430013089078E0194830F9140042
:103B100000EB800001010D480A30005D91FBF0F8D8
:103B2000184830F81400A8EB00000FFA80F810488D
:103B300030F91470144830F9140027E0FC04002018
:103B4000A00100202C0100209C010020AC030020DB
:103B500030010020340100200E02002035FA8E3C96
:103B6000EA010020EE010020000020415201002067
:103B7000B00100200CFEFFFFCC0000208E010020D1
:103B8000F0D8FFFFC000002088010020404410F55D
:103B90007A5F01DA40480DE0404830F914004044B3
:103BA000B0F57A5F02DD4FF47A5003E03B4830F91C
:103BB0001400404400B2394921F81400384830F963
:103BC0001400002803DD364830F9140003E03448BF
:103BD00030F914004042B0F5207F03DD00202F496A
:103BE00021F814002D4830F914007D2190FBF1F0EC
:103BF0002C49095D4843801100B20890284931F9E9
:103C00001410294A125D51430A2291FBF2F0C117A8
:103C100000EB5171A7EBE1010FB2214830F814001D
:103C2000224931F81410401A0FFA80F91C4830F874
:103C300014001E4921F814001D4830F814001D49D5
:103C400031F81410084448440FFA80FA184830F844
:103C50001400184921F81400154820F8149016484B
:103C6000005D00FB0AF040110FFA80FB0898384411
:103C7000A0EB0B0000B2114921F81400601CC4B283
:103C8000032CFFF6C5AEFDF793FEFDF73EFEFDF7F4
:103C900068FE09B0BDE8F08F80C1FFFF88010020F9
:103CA000C0000020C0030020B801002076010020E1
:103CB0007C01002082010020BE010020C201002002
:103CC00010B5F149F14803F0CBF810BD2DE9F047EC
:103CD0000446EF4991F8680004F0D0FC8046204685
:103CE00004F0CCFC8146EB4904F049FC0746EA4964
:103CF00004F07BFC0646414604F041FC054604F016
:103D0000DBFC80B2BDE8F08770B50025002406E03A
:103D100003F060F905440A2002F024FE641C202C04
:103D2000F6D3C5F34F10FFF7D1FF0546022407E095
:103D3000D74890F869006043A84200D902E0641CAB
:103D4000062CF5D300BFD5490C70D14890F86A0015
:103D50006043D349088070BD10B5D2480088002860
:103D600051DD00241CE0CF480088B0F5C87F03D1A6
:103D70000020CD4941F82400CB4850F82400CB491D
:103D800031F914100844C84941F824000020C749FB
:103D900021F814000021BE48303020F81410641CB3
:103DA000032CE0DBBF480088012827D1BE4800680B
:103DB0004FF4C87190FBF1F000B2B5490886BA48DB
:103DC00040684FF4C87190FBF1F001B2B0484186F1
:103DD000B54880684FF4C87190FBF1F0B449098888
:103DE000401A01B2AA4881860020A949C88700214B
:103DF000A748A0F840100120FDF730F8A948008836
:103E0000401EA84908800420FDF7BCF900287DD099
:103E1000A8480088322811D19D48008EA649088004
:103E20009B48408E48809A48808E88809848C08FF2
:103E3000A24908809648B0F8400048809D48008814
:103E4000002846DD00241BE09A480088322803D170
:103E500000209B4941F82400994850F824009349D8
:103E600031F914100844964941F8240000208F4984
:103E700021F8140000218648303020F81410641C0A
:103E8000032CE1DB8B48008801281DD100208D49DF
:103E9000088001208C49088002208C4908708648DF
:103EA00000887B4908868448418879484186824851
:103EB000818877488186814800887549C8877F480E
:103EC00041887348A0F840107A480088401E79491C
:103ED00008807F480088012829D100207C4908807B
:103EE00077480068322190FBF1F000B268490886FB
:103EF00073484068322190FBF1F001B2644841867A
:103F00006F488068322190FBF1F000E00FE06849D3
:103F10000988401A01B25E48818600205C49C88742
:103F200000215B48A0F840100120FCF797FF5F4894
:103F300000885749098E401A00B25C49088008463B
:103F400041885348408E081A00B2584948800846B4
:103F500081884F48808E081A00B25449888010BD6D
:103F600010B54A48416851488847484881684F48D9
:103F70008847FFF7F1FE10BD10B5564800880028AD
:103F800037DD00242EE053480088B0F57A7F03D156
:103F90000020514941F824004F4850F824004F496F
:103FA00031F9141008444C4941F8240000204B49D1
:103FB00021F814004A4921F81400464800880128D5
:103FC0000FD1454850F824004FF47A7190FBF1F07E
:103FD00000B2434921F8140001220F210A20FEF704
:103FE00027FD641C032CCEDB3A480088401E39496B
:103FF0000880002438E0394830F81400384931F896
:104000001410401A00B2354921F81400084630F95E
:104010001410344830F91400A0F54870814205DAD4
:10402000304830F91400A0F5487012E02B4830F900
:1040300014102C4830F9140000F54870814205DD59
:10404000284830F9140000F5487002E0234830F9A0
:10405000140000B2214921F81400084630F8140079
:10406000204921F81400641C032CC4DB10BD10B5DA
:1040700005484168194888470348816817488847B8
:10408000FFF77AFF10BD00007005002060050020DA
:10409000AC0300203333534000F07F45640100201F
:1040A000F4010020F60100203C050020F200002071
:1040B000FA0100205C010020FE0100200402002023
:1040C00048050020620100205E0100202801002038
:1040D00060010020F801002054050020EC000020C1
:1040E000C60000200802002010B50446FE490C70EE
:1040F0000846007802F00DFEFC480078FA4909787D
:104100004840FA490870200AF749087008460078C4
:1041100002F0FFFDF5480078F34909784840F3497B
:104120000870200CF04908700846007802F0F1FD94
:10413000EE480078EC4909784840EC490870200EB8
:10414000E94908700846007802F0E3FDE748007886
:10415000E54909784840E549087010BD10B50446A6
:10416000E3490C700846007802F0D3FDDF48007880
:10417000DF4909784840DD490870200ADC490870A9
:104180000846007802F0C5FDD8480078D84909787B
:104190004840D649087010BD10B50446204602F0CC
:1041A000B8FDD24800786040D049087010BDD148B1
:1041B00001780078401CCF4A1070CF48405C7047AF
:1041C00000B5FFF7F4FF0346FFF7F1FF03EB002014
:1041D00083B2184600BD10B5FFF7F2FF0446FFF7A3
:1041E000EFFF04EB0044204610BD70B504460D46B9
:1041F0002420FFF7D1FF4D20FFF7CEFF0CB1212186
:1042000000E03E210846FFF7C7FF0020B7490870CD
:104210002846FFF7C1FFB9480078FFF7BDFF70BD22
:1042200010B5044621460020FFF7DFFF10BD10B592
:10423000044621460120FFF7D8FF10BD10B5AB485A
:104240000078FFF7A9FF10BD70B505462C4603E0C6
:104250002078FFF7A1FF641C20780028F8D170BDFA
:1042600010B50446204602F090FC10BD2DE9F04147
:10427000A2480078732879D00DDCA0F164000F28E3
:1042800075D2DFE800F0BED1FDFCFBFAF9F8F7F6D5
:10429000F5F4F3F2F100CC287DD010DCC8281DD055
:1042A00006DC742874D0752873D076285FD166E256
:1042B000C92822D0CA2842D0CB28F7D159E0D0282B
:1042C00068D006DCCD287DD0CE287CD0CF28EDD19B
:1042D00093E0FA2878D0FE28E8D19AE2002406E09C
:1042E000FFF76EFF00B2864921F81400641C082C09
:1042F000F6D30020FFF794FF9DE2FFF758FF8149B6
:10430000C872FFF754FF80490870FFF764FF7F49C8
:104310000860FFF760FF7D494860FFF751FF7C4967
:104320000880FFF74DFF7B4908807B48007840F00C
:104330000200794908700020FFF772FF7BE2002439
:104340000EE0FFF734FF75490855FFF730FF73495A
:104350000A310855FFF72BFF704914310855641CCA
:104360000A2CEED30020FFF75BFF64E2FAE15EE285
:1043700011E0002406E0FFF723FF6849423121F8ED
:104380001400641C0E2CF6D30020FFF749FF52E204
:10439000D3E1D9E120E2FFF70AFF60490A3981F849
:1043A0002800FFF704FF5D490A3981F82900FFF76B
:1043B000FEFE5A490A3981F82C00FFF7F8FE5749EA
:1043C0000A3902E00FE216E21CE281F82D00FFF745
:1043D000EEFE52490A3981F82E00FFF7E8FE4F49F8
:1043E0000A3981F82A00FFF7E2FE4C490A3981F8C0
:1043F0002B000020FFF714FF1DE20020FFF710FF45
:1044000019E20720FFF70CFFD220FFF7C5FE434952
:104410000A394878FFF7C0FE0020FFF7BDFE4FF0D5
:104420000040FFF761FE06E20A20FFF7F9FE3C4874
:10443000008800B2FFF792FE02F03FFA06B2304663
:10444000FFF78CFE0120FCF785FE07460220FCF7F3
:1044500081FE47EA40070420FCF77CFE47EA80071C
:104460001020FCF777FE0CE075E156E13DE115E127
:1044700009E100E1E7E0D2E0B3E0A4E095E086E006
:1044800063E047EAC0070820FCF764FE47EA00162D
:104490003046FFF763FE1B4909791A4A927941EACF
:1044A0004201184A527941EA8201164A527841EA99
:1044B00042111C4AD27841EAC2011A4A127941EAF1
:1044C0000211104AD27941EA82110E4A127A41EA67
:1044D000C2110C4A527A41EA42210A4A927A41EACE
:1044E0000221104A927A1FE01402002019020020D3
:1044F000150200201A020020800500201B02002067
:104500003C010020FC040020E0010020C801002044
:10451000E6010020E801002050010020B603002041
:10452000340100202E05002041EA8221FE4AD27A81
:1045300041EAC221FC4A127B41EA0231FA4A527B2B
:1045400041EA4230FFF7D0FD75E11220FFF768FE27
:10455000002405E0F54931F91400FFF7FFFD641C64
:10456000032CF7D3002405E0F14931F91400FFF7DB
:10457000F5FD641C032CF7D3002405E0ED4931F967
:104580001400FFF7EBFD641C032CF7D353E110205C
:10459000FFF746FE002405E0E74931F91400FFF774
:1045A000DDFD641C082CF7D345E11020FFF738FE31
:1045B000002405E0E14931F91400FFF7CFFD641C48
:1045C000082CF7D337E11020FFF72AFE002405E07E
:1045D000DB4931F91400FFF7C1FD641C082CF7D347
:1045E00029E10E20FFF71CFED649C87AFFF7D4FD5B
:1045F000D5480078FFF7D0FDD4490868FFF774FD6F
:10460000D2494868FFF770FDD148008800B2FFF733
:10461000A5FDD048008800B2FFF7A0FD0BE1052002
:10462000FFF7FEFDCC48008800B2FFF797FDCB48AE
:10463000B0F90000FFF792FDC949097801F00100C7
:10464000FFF7AAFDF7E00820FFF7EAFD002405E0E8
:10465000C44931F91400FFF781FD641C022CF7D323
:10466000C148B0F90000FFF779FDC048B0F900007B
:10467000FFF774FDDFE00420FFF7D2FDBC480068BF
:10468000FFF732FDD7E00320FFF7CAFDB9480078F5
:10469000FFF782FD0020FFF761FDCCE00720FFF768
:1046A000BFFDB54991F82800FFF776FDB24991F8B2
:1046B0002900FFF771FDB04991F82C00FFF76CFD60
:1046C000AD4991F82D00FFF767FDAB4991F82E0039
:1046D000FFF762FDA84991F82A00FFF75DFDA649A2
:1046E00091F82B00FFF758FDA5E01E20FFF798FD7D
:1046F00000240FE0A0490A31085DFFF74DFD9E49F7
:104700001431085DFFF748FD9B491E31085DFFF736
:1047100043FD641C0A2CEDD38DE01C20FFF780FDC7
:10472000002407E094494C3131F8141008B2FFF727
:1047300015FD641C0E2CF5D37DE06320FFF770FDA2
:104740008E48FFF781FD76E02F20FFF769FD8C484A
:10475000FFF77AFD6FE00220FFF762FD0020FFF710
:10476000FDFC68E00820FFF75BFD002404E0601C0E
:10477000C0B2FFF711FD641C082CF8D35BE0FFF713
:1047800016FD05460C20FFF74BFD8DB90020FFF705
:1047900003FD7C490868FFF7A7FC7A494868FFF7E2
:1047A000A3FC0020FFF7DAFC0020FFF7F5FC12E085
:1047B000102D10D11020FFF7EFFC73490868FFF7A8
:1047C00093FC71494868FFF78FFC0020FFF7C6FC97
:1047D0000020FFF7E1FC2EE00120FCF774FB002035
:1047E000FFF71EFD27E04FF4C870684908800020DD
:1047F000FFF716FD1FE00120524988730020FFF7E4
:104800000FFD18E00020FCF729FB0020FFF708FD52
:1048100011E00820FFF704FD002405E05C4931F9B0
:104820001400FFF79BFC641C042CF7D303E000206A
:10483000FFF7FDFC00BF00BFFFF700FDBDE8F08102
:1048400010B50446232C02D0522C07D102E0FCF70D
:1048500064F803E0012002F033F900BF00BF10BD8F
:1048600010B54C48007810B1FCF757F810BDCDE0FA
:1048700002F036FA04464848007870B9242C01D179
:10488000012000E000204449087008460078002814
:1048900002D12046FFF7D4FFB7E03F480078012857
:1048A00007D14D2C01D1022000E000203A490870C8
:1048B000ABE039480078022807D13C2C01D1032015
:1048C00000E00020344908709FE033480078032856
:1048D0001AD1402C03DD00202F49087096E02F48A4
:1048E000047000202E4908702E4908702E49087067
:1048F0002C48007860402B49087004202649087035
:1049000001202A49087080E023480078042851D10A
:104910002748047023480078604022490870052029
:104920001D49087071E000002E050020F8000020ED
:10493000C0000020FE000020160100208C04002092
:104940003C010020FC040020E0010020C801002000
:10495000E6010020E8010020E2010020E40100203F
:1049600050010020CC0000200E020020AA010020EF
:104970000C010020AC010020AC0300200D970008C2
:1049800071970008D0010020D8010020F601002016
:10499000A2010020130200201802002017020020AC
:1049A00016020020190200201A0200201202002024
:1049B0001B02002021480078052813D120480078E8
:1049C0002049097888420DDA1F48007860401E4966
:1049D00008701B4801780078401C194A10701B4869
:1049E000445412E01548007805280ED11448007888
:1049F00014490978884208DB13480078A04201D1A5
:104A0000FFF734FC00200D49087000BF02F051F997
:104A100000287FF42DAF0E48007868B902F049F9FC
:104A200050B94FF40060FCF7ADFB28B1094840785D
:104A300010B101F02BFB19E700BF17E718020020A7
:104A40001602002017020020190200208005002015
:104A500013020020FC04002044F25061884201DD72
:104A6000A0EB4100FA49884202DA48F6A041084426
:104A7000704700B5F7480068F7490968421A1046C0
:104A8000FFF7EAFF0246002A01DD104600E050422F
:104A900042F21071884201DD012000BD0020FCE7D8
:104AA000014608687047016070472DE9FE4F0446D3
:104AB0000E4615461F466168701A03F0D6FD804603
:104AC000296803F092FD2061A168206903F051FD7F
:104AD000E249029091F8AE0003F0D0FDE049009069
:104AE00003F04DFD014601904FF07E5003F07DFD37
:104AF0008346296803F0EBFC82465146286803F0A0
:104B000074FD8146029903F03AFD8046A16803F0E6
:104B1000DEFC206166602069A0602169B86803F04E
:104B20002EFD804603F0AFFDBDE8FE8F2DE9F04776
:104B300004460E4617461D46304603F096FD824653
:104B4000696803F01CFD8146396803F018FD804652
:104B5000216803F0BCFC2060E86880F00048404613
:104B6000216803F0C7FD04D2E86880F000402060AF
:104B700006E0E968206803F0BDFD01D2E868206026
:104B8000206803F080FDBDE8F0872DE9F041804604
:104B90000C461546204603F068FD0746296803F0D9
:104BA000EEFC064603F06FFDBDE8F08148F6A0413B
:104BB000884200DD401A002802DA48F6A041084485
:104BC00070472DE9F041A3490968A34A1268881A81
:104BD000FFF742FF002807DD9E4909689E4A1268D8
:104BE000881AFFF739FF07E09A4909689A4A12685C
:104BF000881AFFF731FF404241F2941188423DDAB2
:104C000094490968944A1268881A03F02EFD0546F3
:104C1000944903F0B4FC04469349086803F02EFD60
:104C20000646204604F0A4F90746314603F0A7FCE7
:104C3000054603F028FD00B28C4908800846B0F90B
:104C400000008B49884201DA08460BE08748B0F93A
:104C5000000040F6B831884201DD084602E0834892
:104C6000B0F900007B490968084482490860084699
:104C70000068FFF79BFF7F49086003E07548006804
:104C80007C490860BDE8F0812DE9FC470546FFF747
:104C900098FF7849096842F22832501A03F0E5FC7F
:104CA0000746704903F06BFC0646304604F0A0F856
:104CB0000190304604F05CF90090002481E06E49D8
:104CC00031F9140003F0D1FC8146284603F0CDFCF5
:104CD00082465DF8241003F052FC8046494603F0FA
:104CE00048FC074603F0CFFC00B2644921F81400E9
:104CF000084630F9140010F57A7F01DA60480BE0BD
:104D00005E4830F91400B0F57A7F02DD4FF47A7016
:104D100002E05A4830F91400584921F814000A46B4
:104D200032F9141004EB8402564B03EB8200564A0E
:104D3000FFF72BFF0746514A32F9141004EB8402A7
:104D4000504B03EB8200504B504AFFF7EFFE0744F5
:104D50004A4A32F9141004EB84024A4B03EB8200F6
:104D6000494B4A4AFFF7A1FE384400B2484921F8AE
:104D70001400084630F914003D49884201DA08461B
:104D80000BE0434830F9140040F6B831884201DDA9
:104D9000084602E03E4830F914003D4921F814006D
:104DA00004EB8401374A02EB8100FFF779FE0746E6
:104DB00004EB8401374A02EB81003946FFF773FEAA
:104DC000641C022CFFF67BAFBDE8FC8770B504467F
:104DD0000D468DB124480068B4EB500F01D2204637
:104DE00002E021480068400804B2002C01DD2046A2
:104DF00000E00020044613E01B480068844201D212
:104E0000204601E01848006804B21448B0F8B20027
:104E1000A04201DA204602E01048B0F8B20004B225
:104E20001D48B0F90000844210DD184801681B4895
:104E300003F0A5FB064603F026FC17490988084441
:104E400000B2154908800846B0F90040204670BD00
:104E5000B0B9FFFF580200205C020020AC03002024
:104E6000DB0FC940D3023739640200206002002002
:104E700048F4FFFF900200201C02002044020020A2
:104E800018FCFFFF50060020F00500203C02002027
:104E9000EA01002028060020680200200000C84225
:104EA0002DE9F04700247DE0FA4A52F8241004EB83
:104EB0008402F94B03EB8200F84AFFF766FE814655
:104EC000F74830F81400A9EB000000B2F54921F8CA
:104ED00014000A4632F9141004EB8402F24B03EB7F
:104EE0008200F24AFFF751FE0746EE4A32F91420DB
:104EF000E84B53F82430D11804EB8402EA4B03EB5F
:104F00008200EA4BEA4AFFF711FE8046E14A52F876
:104F1000241004EB8402E44B03EB8200E34BE44AED
:104F2000FFF7C3FD054615F5FA6F01DAE14806E023
:104F3000B5F5FA6F02DD4FF4FA6000E02846054649
:104F4000D74830F91400002803DDD54830F91400A3
:104F500003E0D34830F914004042322800DA00253B
:104F600007EB08004619D448864200DA05E040F60F
:104F7000B830864200DD00E0304600B2CF4921F86B
:104F8000140004EB8401C84A02EB8100FFF788FD9E
:104F9000824604EB8401CA4A02EB81005146FFF7C6
:104FA00082FD641C022CFFF67FAFBDE8F0872DE97F
:104FB000F04704460D4616461F4629683A68881A87
:104FC00003F053FB8146BF480168484603F0D7FA17
:104FD000804603F058FBAF49486020683168401AAA
:104FE000AC490860BDE8F0872DE9FF5F06460F4633
:104FF000904699460F9CD8F800103268881A03F042
:1050000034FB0546D9F800103A68881A03F02DFBE6
:105010008346AC480168584603F0B1FA82465146CF
:10502000504603F0ACFA29460190284603F0A7FA4F
:105030000090019903F04BFA029004F05FF8A24946
:10504000039003F09CFA834603F036FB0E99086048
:1050500085F0004B5146584603F0A0FD9B49019056
:1050600003F08DFA9A49029003F031FA039003F0AD
:105070000AFB20602068002804DA48F6A041206876
:1050800008442060BDE8FF9F2DE9F0419148007879
:1050900000284FD0864801684FF07E5003F0A5FAF3
:1050A00006468D4949688D4A5268881A03F0DDFA30
:1050B000074684480168384603F061FA05463146E0
:1050C00003F05DFA044603F0DEFA00B2744948804A
:1050D00081490968814A1268881A03F0C6FA0546B0
:1050E000314603F04CFA044603F0CDFA00B26C49A5
:1050F0000880B1F902107A4AB2F90220881800EB50
:10510000D071491009B2664A51801146B1F90010B8
:10511000734AB2F90020881800EBD071491009B227
:105120005F4A1180104640886D49488010460088CB
:10513000088000BF012067490870674840686749D8
:105140004860654800680860BDE8F0812DE9F041DD
:105150000546284603F089FA0746002103F0CAFAFB
:1051600003D2284603F081FA04E0284603F07DFAD2
:1051700080F0004006465B4903F001FA04462046F1
:1051800003F036FE4F490860BDE8F081A0F1300120
:10519000C8B2092801DDC11FC8B200F00F00704776
:1051A00030B502460B460020002115E0545C2E2C41
:1051B00005D1491C03B912E00024CD18545500EB69
:1051C00080046000545C302C05DB545C392C02DC1C
:1051D000545C303C2044491C545C002CE6D100BF98
:1051E00030BD2DE9F047804600260027B1464546F0
:1051F00000E06D1C03F0CCF800682978405C2028A2
:10520000F7D0444609E01EB106EB86004006060EC4
:1052100014F8010B30383044C6B2281B0228F2DCE7
:1052200009E01FB107EB87004006070E14F8010BD9
:1052300030383844C7B2A542F3D828782E2817D181
:105240006C1C4FF0000A10E009EB89004FEA40099E
:1052500003F09EF800682178405C202803D114F800
:10526000010B303881440AF1010ABAF1040FEBDB7B
:105270001D48784309EBC90101EB091100EB8100DE
:105280000621B0FBF1F11948704301EBC010BDE8F5
:10529000F08700004802002000060020D005002012
:1052A0001C0200204402002028060020E005002007
:1052B0003C02002030F8FFFF48F4FFFFEA01002025
:1052C00050060020400200202C7D8E3FA00CB345EC
:1052D00000A00C4634020020C80100202C0200204F
:1052E0002802002050E0EF3040420F002D31010035
:1052F00070B504460026242C07D10020FE49087012
:10530000FE490870FE490870F1E02C2C01D02A2CCF
:1053100077D10020FB49F94A12788854F648007882
:1053200080BB0020F8490870F6480078472811D162
:10533000F448407850280DD1F2488078472809D1A8
:10534000F048C078472805D1EE480079412801D1BE
:1053500001200870EB480078472812D1E9484078CE
:1053600050287ED1E748807852287AD1E548C07825
:105370004D2876D1E3480079432872D10220E249D2
:1053800008706EE0FFE7E0480078012854D1DA4861
:105390000078022805D1DB48FFF723FFDB490860CE
:1053A0005FE0D5480078032809D1D6480078532813
:1053B00005D1D64800684042D449086051E0CE4843
:1053C0000078042805D1CF48FFF70BFFCF4948608C
:1053D00047E0C9480078052809D1CA48007857280D
:1053E00005D1CA4840684042C849486039E0C248CF
:1053F000007806280AD1C3480078302802DD012051
:1054000001E042E00020C249C8722AE0BA480078B0
:10541000072806D10021BB48FFF7C2FEBD4908702E
:105420001FE0B548007809281BD10021B548FFF7D7
:10543000B7FEB949088014E0B3480078022810D1BB
:10544000AD48007807280CD10121AE48FFF7A8FE2F
:1054500041F2184148434FF47A71B0FBF1F0AF4983
:105460000880A5480078401CA34908700020A34983
:1054700008702A2C03D10120A949087037E0A04800
:10548000007860409E49087031E00D2C01D00A2C54
:1054900019D1A348007890B19A490878FFF776FEB1
:1054A00005462807050E97494878FFF76FFE284400
:1054B000C5B293480078854200D1012600BF002084
:1054C0009749087013E08D4800780F2807DA8B4859
:1054D00001780078401C894A10708A4844549048EA
:1054E000007820B986480078604085490870864871
:1054F000007810B101208B49087026B182480078ED
:10550000012800D170BD0020FCE72DE9FF410546D0
:10551000E8B2FFF7EDFE00287ED08348007801282E
:1055200003D100208049087002E001207E49087004
:105530007748C07A0028EFD07648007805286BDBE2
:105540007348407810B90020714908737048007B97
:10555000A8B96F48407890B101206D4908736B4835
:10556000006872490860694840684860674908688F
:10557000FFF7ECFD6E48B0F900006E4908806E48F8
:105580000078401C052190FBF1F201FB12006A49F2
:10559000087000247AE05D4850F82400674941F81B
:1055A0002400084650F82400654990FBF1F0654955
:1055B00041F82400614850F82410624850F8240053
:1055C000614A5043A1EBC01042F2107190FBF1F020
:1055D0005E4921F8140004EB84005D4901EB800072
:1055E0005549097850F821005A4951F82410081AF1
:1055F000584941F82400514850F82410514850F8B7
:1056000024005043A1EBC01004EB8401504A02EB8C
:105610008101494A127800E0FFE041F8220004EBE2
:1056200084004B4901EB80004349097850F8210080
:10563000484951F824100844464941F824000846D6
:1056400050F82400052190FBF1F13E4850F8240069
:105650003D4A504301EBC0103F4941F824003F4808
:105660000078012811D1394830F8140001280CDDE8
:10567000364830F8140040F2E731884205DA3648FF
:1056800050F82400214941F82400641C022C82DBDC
:1056900001F059F932490968471A384602F0EEFF1D
:1056A0000646304902F0A1FF2F49086001F04BF98E
:1056B0002B4908604FF07E512B48006803F010F82A
:1056C00002D22948006801E04FF07E502649086068
:1056D00002A803A9154B1B1D1A1FCDE900100B4989
:1056E000091D081FFFF780FC64210398B0FBF1F04F
:1056F0001E49088064213BE035020020360200206C
:1057000037020020C005002039020020C801002017
:10571000FC040020E0010020E6010020E801002058
:10572000380200205801002050010020D001002044
:105730000E020020940200202002002074020020AB
:1057400080969800840200202D3101008C020020F8
:10575000780600206C0200207C0200205A01002004
:105760002402002000007A443C020020E2010020D4
:10577000029890FBF1F000B295490880FFF784FC95
:105780009448007A18B99348C079002845D09248C7
:105790009249934B1A1FCDE900109249081FFFF759
:1057A00023FC904B1A1F8E49081FFFF700FC8E4800
:1057B00090F90000012802D002282DD102E0FFF765
:1057C0006FFB29E08949B1F8B41008B20121FFF755
:1057D000FDFA80464046FFF757FA844890F8B0003B
:1057E00038B183480068642190FBF1F000B2814930
:1057F00008807E48B0F8AC0078490968884202D237
:10580000FFF737F938B10120774908707A48B0F9C5
:1058100000007849088000BF00BFBDE8FF8110B5D7
:105820007249887B02F02AFF0446744902F0DDFECB
:10583000734908606D49087E02F020FF04466F49F5
:1058400002F0D3FE6E4948606E48C8606749C87B65
:1058500002F014FF04466C4902F0C7FE6B49086071
:105860006249487E02F00AFF0446644902F0BDFE28
:10587000664948605D4991F8230002F0FFFE044646
:10588000634902F0B2FE614988605E48C8605749CA
:10589000087C02F0F3FE04465B4902F0A6FE5D4977
:1058A00008605249887E02F0E9FE0446534902F03E
:1058B0009CFE584948604D4991F8240002F0DEFEF4
:1058C0000446534902F091FE524988604D48C86031
:1058D00010BD10B50446FFF7A2FF4F49204601F066
:1058E00037FA4FF4FA7001F03DF84C48007810B1E7
:1058F0001020FBF738FC10BD002101604160816081
:1059000070473448C07AA0B145480078052810DBBC
:105910003448001F0068434908603248001F40684F
:1059200048604148B0F90000334908800120294906
:105930000873704710B500241CE000203B4921F893
:1059400014003B4921F8140004EB8401394A02EBAE
:105950008100FFF7D1FF04EB8401374A02EB81009D
:10596000FFF7CAFF04EB8401344A02EB8100FFF722
:10597000C3FF641C022CE0DB10BD7CB504460D4661
:105980001749091F20680860286848602068FFF7E9
:10599000DDFB11481149124B1A1FCDE900101149C6
:1059A000081FFFF721FB0C480068114908600D4BE8
:1059B0001A1F0B49081FFFF7FAFA07480068204929
:1059C00008600A48B0F8B20000B21E4908807CBDE9
:1059D000E4010020FC0400205802002064020020A2
:1059E00054020020CC0100205A010020AC0300200A
:1059F0009002002010020020940200200000C84203
:105A0000D00500200000FA4400002041E0050020FD
:105A100000007A44F00500200B55000858010020D2
:105A2000E0010020D00100200E02002052010020E1
:105A3000EA01002000060020280600205006002071
:105A40005C0200206802002070B50446012046492F
:105A5000087000F062FF054644480068281A44496F
:105A60000860424805600846006841F28831884273
:105A700002D900203F4908703F493E4A12788C54B1
:105A80003C4800780F2806D101203C4908700020CE
:105A90003B49088004E037480078401C35490870CD
:105AA00070BD10B5374890F8760030B10320364904
:105AB000087007203549087005E002203249087057
:105AC00003203249087032494FF4E13001F040F9C7
:105AD00010BD2A480078704770B50246274B1B78E6
:105AE000FBB1032118E04C1E234D2C5D264D2D7873
:105AF0002C4104F00F03072B0CDA1F4C655C4C1E85
:105B00001D4E345D214E3678344005EB0424214D82
:105B100045F823408B1CD9B21029E4DB0023174C35
:105B20002370072A02DA104B1B781BB9154BB3F808
:105B3000780018E0134B93F876305BB1114B6B3360
:105B40009B5C144C54F823304FF4777404EB5303EC
:105B500098B208E00B4B6B339B5C0E4C54F823302F
:105B600003F5777398B270BD990200209C02002063
:105B7000A0020020A4020020BC0600209802002001
:105B800038010020AC030020A5020020A60200205E
:105B9000495A0008A006002010B50446A048007825
:105BA00070B900F0D0FE9F4909683231884207D3AE
:105BB00001209B49087000F0C6FE9A4908601CE06D
:105BC00097480078C8B100F0BEFE964909682144A4
:105BD000884212D300209249087000F0B4FE914927
:105BE000086091480078002804DD8F480078401E46
:105BF0008D49087001208D49087010BD2DE9F843CA
:105C000005460E46174698468DF800508DF80160FF
:105C10008DF802708DF80380854909781DF8010020
:105C200044280AD04C2806D04D2802D04E2809D14D
:105C300006E0642408E0C82406E04FF4FA6403E0B8
:105C4000002401E0322400BF00BF79480078032817
:105C500003DA14B12046FFF79FFF75480078032848
:105C60000BDB00F070FE001B6E490968884204D906
:105C700000206F4908706C4908706C480078012852
:105C800000D06CB96A480078032804DA68480078C4
:105C9000401C67490870002064490870604908701A
:105CA000BDE8F88310B504466248807A18B1012037
:105CB0006149087002E000205F4908704FF40070ED
:105CC000FBF760FAB0B35D4890F87F0000EB80000E
:105CD0005B49B1F90010884216DA5A48407898B109
:105CE000012059490870554890F87F00534991F8B0
:105CF0008010084400EB80005149B1F9001088423F
:105D000002DA0220504908704C4890F87F0000EBFE
:105D100080004B49B1F90010884205DA49484078C3
:105D200010B90220484908704548008810B9002081
:105D3000454908701020FBF70DFA78B13D4880798D
:105D400010B93C48C07930B13E48C07A18B901203A
:105D50003E49087002E000203C4908703A4800784B
:105D6000022806D144234E2211464C20FFF746FF5D
:105D700054E035480078012806D14D234C221946BD
:105D80005320FFF73BFF49E030480078012806D157
:105D90004D234E2253210846FFF730FF3EE02648B0
:105DA0000078012806D14D23532211461046FFF7F3
:105DB00025FF33E0042C06D144234D221146532005
:105DC000FFF71CFF2AE0022C06D144234D22532169
:105DD0000846FFF713FF21E0012C06D144234E2291
:105DE0004D215320FFF70AFF18E0194800780128D9
:105DF00009D11448407830B14E234D225321084632
:105E0000FFF7FCFE0AE008480078002803DD322096
:105E1000FFF7C2FE02E000200149087010BD00003B
:105E2000A8020020B002002028010020A9020020C2
:105E3000AE0200202E050020AA020020AC030020A4
:105E400038010020FC040020AC020020AB0200203E
:105E5000AD02002010B504465E2000F05AFF204637
:105E600000F057FF10BD10B55E2000F052FF10BDCE
:105E700070B50446E5B2284600F04BFFC4F3072591
:105E8000284600F046FF70BD2DE9F04700241FE0D2
:105E900004F12401C8B2FFF7DDFF9748008802F043
:105EA000EDFB8046954931F9140002F0DEFB814696
:105EB000414602F09AFB0746914902F060FB064614
:105EC00002F0E1FB05B22846FFF7D2FF601CC4B226
:105ED000032CDDDBBDE8F08710B51020FFF7BAFF1B
:105EE00088480068642190FBF1F004B22046FFF777
:105EF000BFFF2120FFF7AEFF82480068642190FBBE
:105F0000F1F201FB120004B22046FFF7B1FF10BD11
:105F100010B50220FFF79EFF7B48B0F900000A2170
:105F200090FBF1F004B22046FFF7A2FF10BD70B560
:105F300000F009FD4FF47A71B0FBF1F43C20B4FBA2
:105F4000F0F03C21B0FBF1F201FB12051720FFF746
:105F500081FF290208B2FFF78BFF1820FFF77AFFB5
:105F60003C20B4FBF0F100FB114006B23046FFF7D5
:105F70007FFF70BD10B51320FFF76CFF634800680A
:105F8000002802DD6148006802E060480068404285
:105F90005F4990FBF1F004B22046FFF769FF1B2038
:105FA000FFF758FF59480068002802DD574800688D
:105FB00002E0564800684042554990FBF1F042F239
:105FC000107190FBF1F201FB120004B22046FFF7C2
:105FD0004FFF2320FFF73EFF4C490968002901DAF3
:105FE000532100E04E210846FFF742FF1220FFF741
:105FF00031FF46484068002802DD4448406802E01E
:10600000424840684042424990FBF1F004B22046C9
:10601000FFF72EFF1A20FFF71DFF3C4840680028BD
:1060200002DD3A48406802E038484068404238495A
:1060300090FBF1F042F2107190FBF1F201FB1200C3
:1060400004B22046FFF714FF2220FFF703FF2F4979
:106050004968002901DA572100E045210846FFF789
:1060600007FF10BD10B504462A48007884420CD0C2
:1060700024B14FF41650FEF7F3F804E02649D1F8A6
:10608000B800FEF7EDF82348047010BD10B500F01D
:106090005AFC22490968401AC8282BD300F053FC47
:1060A0001E4908601E480078401C1D490870FFF713
:1060B000EBFEFFF711FFFFF72BFFFFF7D4FE1848A9
:1060C0000078052190FBF1F201FB120038B9102095
:1060D000FBF740F818B1FFF74DFFFFF7C4FE10487B
:1060E0000078192806D100200D490870FFF71FFF1E
:1060F000FFF7B9FE10BD0000FA010020F8000020F3
:1061000000007A440C010020AE010020C8010020EC
:10611000A0860100B4020020AC030020B8020020D9
:10612000BC02002038B54FF44060ADF800000220FA
:106130008DF8020014208DF803006946FA4801F03A
:10614000CDFF4FF44061F84802F021F800241CE034
:1061500002E00A2000F0FAFB4FF48061F24802F0FE
:106160000FF80028F5D04FF48061EF4802F011F8E5
:106170000A2000F0EBFB4FF48061EB4802F007F8D7
:106180000A2000F0E3FB601CC4B2082CE0DB4FF4F3
:106190000061E54801F0FDFF0A2000F0D7FB4FF455
:1061A0008061E14801F0F5FF0A2000F0CFFB4FF4D9
:1061B0008061DD4801F0EBFF0A2000F0C7FB4FF4DF
:1061C0000061D94801F0E3FF4FF44060ADF80000F2
:1061D00002208DF802001C208DF803006946D24889
:1061E00001F07CFF38BD10B586B004464FF4406026
:1061F000ADF8100002208DF812001C208DF813005D
:1062000004A9C94801F06AFFC8480460FFF78AFF83
:10621000C648006801F00EFB684601F076FB0022DC
:106220004FF44071C148006801F0A5FB0020ADF8B3
:1062300004004BF6FF70ADF806004FF48040ADF857
:106240000C00BB4800900121B848006801F06BFBCE
:106250006946B648006801F000FB4FF4A06001F009
:106260006FF922208DF8140000208DF815008DF8AC
:10627000160001208DF8170005A801F066F921200D
:106280008DF8140000208DF8150005A801F05DF9C7
:1062900006B010BD70B5A5480068848A00BF14F42C
:1062A000E06F3CD0A1480068058B00224FF480616C
:1062B0009E48006801F05FFB14F4007F2FD19B48DB
:1062C0000068008810F4007F29D198480068008891
:1062D00010F4807F17D000BF94480068008810F445
:1062E000807FF9D101219148006801F030FB00BFA7
:1062F0008E480068008810F4007FF9D18B48006850
:10630000FFF771FF0BE001218848006801F01FFBD7
:1063100000224FF440718548006801F02CFB83484F
:106320000068808A20F470608049096888820020B3
:106330008049087070BD10B5FFF7ACFF10BD70B597
:106340007A480068808AC4B214F0010F3FD07748C1
:106350000068008820F40060744909680880012101
:106360007248006801F0FDFA002073490870734814
:106370000078E8B17248007818B972480078FF28B0
:1063800016D101206E4908706F480078022807D1A5
:1063900066480068008840F4006064490968088025
:1063A00001226A4801786148006801F0F1FA98E139
:1063B0000022664801785D48006801F0E9FA61480A
:1063C0000078FF28F3D0FF205B49087089E114F0C2
:1063D000020F5BD0BFF3508F5B48007801281FD1BC
:1063E00056480078E0B156480078C8B100214F48BF
:1063F000006801F0B6FABFF3508F4C480068008B7C
:10640000C5B201214948006801F0A1FA01205049B4
:106410000870012281024548006801F0ACFA34E0BE
:1064200042480068008BC5B2BFF3508F46480078E1
:10643000022812D14148007878B14148007860B113
:1064400000213A48006801F08CFA00224FF4806184
:106450003648006801F08FFA17E03B4800780328BF
:106460000DD13648007850B13548007838B1002257
:106470004FF480612D48006801F07DFA05E00122AB
:1064800091022A48006801F076FA2AE114F0040F1C
:1064900049D001202E4908702848007800287DD076
:1064A00027480078002879D027480078022831DD75
:1064B00000211E48006801F054FA1C48006801F0F1
:1064C00064FA1D4991F900200978491C49B21A4B18
:1064D000197020490968885401211448006801F0A6
:1064E00036FA01201A4908701048006801F04DFA88
:1064F000114991F900200978491C49B20E4B1970D5
:10650000144909688854012291020848006801F082
:1065100032FA70E00E480078F0B1012103480068BB
:1065200001F015FA1DE06EE0000C0140C8020020E9
:10653000801A0600CC020020C5020020D1020020F3
:10654000C3020020CE020020CF020020CD02002096
:10655000C4020020D80200200121D948006801F0BF
:10656000ECF9D748006801F010FAD64991F90020FB
:106570000978491C49B2D34B1970D349096888542A
:10658000CF48006801F001FACE4991F9002009785E
:10659000491C49B2CB4B1970CB4900E008E00968AF
:1065A000885418460078401C40B21946087022E012
:1065B000C648007810B9C6480078A0B1C548007830
:1065C00028B10121BE48006801F0C1F904E00121B1
:1065D000BB48006801F0B1F9BA480078401C40B2ED
:1065E000B849087007E00121B548006801F0A5F935
:1065F0000120B649087000BFB1480068008810F457
:10660000807FF9D16DE014F0400F2BD0AC480068CA
:1066100001F0BBF9AB4991F900200978491C49B256
:10662000A84B1970A84909688854AB4801781846E6
:1066300090F90000C01C814206D100224FF4806115
:106640009F48006801F097F9A34800789D4991F9A7
:106650000010884245D19B480078401C40B29949BF
:1066600008703EE014F0800F3BD0964890F900008F
:10667000401C1DD0934890F900200078401C40B287
:10668000904B187095480068815C8D48006801F057
:106690007AF9914800788B4991F90010884220D10D
:1066A00000224FF480618648006801F064F918E028
:1066B00084480078401C40B28249087088480178BC
:1066C0007F48006801F05FF98648007810B9824879
:1066D000007830B900224FF480617948006801F0F9
:1066E0004AF9784890F900107B480078401C8142B4
:1066F0000FD10020754908707648007830B100222B
:106700004FF440716E48006801F035F90020764979
:10671000087070BD10B5FFF712FE10BD10B5FFF781
:10672000B9FD10BD10B5FFF70AFE10BD2DE9FF47FA
:1067300006460F461546984647F230597006000E39
:106740006A49087066480770012061490870002096
:10675000644908706149C1F800D05B49C1F800D0B4
:106760005D480570012060490870102D03DD002090
:1067700004B0BDE8F087002405E018F804000DF827
:106780000400601CC4B2AC42F7DB4D48006880884E
:1067900010F4007F18D14A480068008810F4807F08
:1067A0000BD100BF46480068008810F4007FF9D183
:1067B00001214348006801F0C0F801224FF4407104
:1067C0003F48006801F0D7F800BF4748007820B183
:1067D000A9F101005FEA0009F7D1B9F1000F0AD170
:1067E00043480088401C4249088035480068FFF74C
:1067F000FAFC0020BCE70120BAE737B504460D4695
:1068000002AB012229462046FFF790FF3EBD2DE94D
:10681000F04105460E4617461C4647F230586806BA
:10682000000E324908702E48067000202849087072
:1068300001202C4908702448046028480460264838
:1068400007700120284908701D480068808810F4EE
:10685000007F18D11A480068008810F4807F0BD19F
:1068600000BF17480068008810F4007FF9D10121AB
:106870001348006801F061F801224FF4407110489C
:10688000006801F078F800BF1748007820B1A8F13F
:1068900001005FEA0008F7D1B8F1000F0BD11448EE
:1068A0000088401C1249088005480068FFF79BFCDF
:1068B0000020BDE8F0810120FBE70D48008870470B
:1068C000C8020020C5020020D8020020C302002018
:1068D000D0020020C4020020CF020020D4020020F9
:1068E000CE020020D1020020CC020020CD020020E8
:1068F000C002002000B585B0684601F057F8754920
:106900000098B0FBF1F07449086005B000BD734811
:106910000068401C71490860704700BF6F480168FB
:106920004FF0E02082696D4800688142F6D16C48E2
:10693000801A4823B0FBF3F001EB4103C3EBC11312
:1069400000EBC300704765480068704730B50446E7
:10695000FFF7E3FF054600BFFFF7DFFF401BA04244
:10696000FAD330BD10B5044603E04FF47A70FFF758
:10697000EDFF2000A4F10104F7D110BDF0B585B002
:10698000584B0FCB8DE80F0002250121564801F02E
:1069900064F8012144F61D2001F056F80121084653
:1069A00001F049F801F06BF84FF6FF70ADF81000F8
:1069B00000208DF8130004A94C4801F08FFB04A9B6
:1069C0004B4801F08BFB04A94A4801F087FB0121E9
:1069D000494801F0E0FB002414E0684600EBC400E5
:1069E0008088ADF8100002208DF81200684600EB98
:1069F000C40080798DF813005DF8340004A901F01B
:106A00006DFB641CAC42E8D34FF4805039490861F7
:106A1000C000364910310860FFF76CFF3748006846
:106A20004FF47A72B0FBF2F1B1F1807F00D31DE038
:106A300021F07F40401E4FF0E022506150170F229E
:106A4000002807DA13071F0E2D4B00F00F06361F24
:106A50009F5503E013071E0E2A4B1E5400BF002053
:106A60004FF0E02290610720106100BF00F026FA8D
:106A70006420FFF777FF05B0F0BD04464FF40040F7
:106A80001A4914310860C0101A49086117E0174804
:106A90000C30006880F4004014490C31086015483F
:106AA000C06880F480501349C86040F2DB1204FBD8
:106AB00002F1881EFFF756FF1920FFF753FFE6E7A4
:106AC00010B11149114A116011490D4A0C3A116077
:106AD0007047000040420F00DC020020E00200206E
:106AE00040190100A4970008070040000008014079
:106AF000000C014000100140000230006003002043
:106B000018ED00E000E400E0EFBEADDEF04F002045
:106B10000400FA0510B5B848B84909680844B849EE
:106B20000865B8480068B549096888420BD9B54876
:106B30000068B2490968401AB1498864B1480068E0
:106B4000AE49086008E0AD480068C0F58070AC4907
:106B500088640020A94908600121A948443000F058
:106B600045FE10BD10B54FF4005000F055FE002159
:106B7000A348443000F03AFEA24800689F490968E3
:106B8000884201D0FFF7C6FF10BD10B592B0044691
:106B90004FF40070ADF8440002208DF84600182034
:106BA0008DF8470011A9984801F098FA4FF48060D9
:106BB000ADF8440048208DF8470011A9924801F033
:106BC0008DFA0E208DF8040001208DF805008DF857
:106BD00006008DF8070001A800F0B7FC0D94002016
:106BE000ADF83800ADF83A00ADF83C00ADF8400023
:106BF0000C20ADF83E000DA9844801F0C7F980488B
:106C0000583000F069FD4FF480500B9000200C903C
:106C10007E48001D02907E4803900020049006905C
:106C2000089080200790002009904FF48070059014
:106C300020200A9002A97248583000F0BAFD0121C4
:106C40006F48583000F0D2FD012240216F4801F01A
:106C500017FA6B48583000F0DCFD6E490860684850
:106C6000443000F039FD6948001D02901020049066
:106C700000200690089080200790002009900A903C
:106C800002A95F48443000F094FD012202215C48D3
:106C9000443000F0B6FD002059498864012280216B
:106CA0005A4801F0EDF90121584801F0C7F912B036
:106CB00010BD10B55248583000F0ABFD5549096879
:106CC000884201D0012010BD0020FCE74B4800683D
:106CD0004C490968884201D1012070470020FCE737
:106CE0004C490968C1F58071494A505C49490968B5
:106CF000491E484A116002D14FF4807111607047FB
:106D000010B500BFFFF7D5FF0028FBD0FFF7E8FF65
:106D100010BD10B5044638483A490968445439480A
:106D20000068401CC0B2374908603548406C10F01C
:106D3000010F01D1FFF7EEFE10BD10B5044603E0D0
:106D400014F8010BFFF7E5FF20780028F8D110BDFB
:106D500030B587B004460D460121480400F07DFEA1
:106D600026208DF8180001208DF8190002208DF8DA
:106D70001A0001208DF81B0006A800F0E6FB082091
:106D8000ADF8140004208DF8170005A91E4801F085
:106D9000A5F901940020ADF80800ADF80A00ADF89F
:106DA0000C000420ADF80E000020ADF8100001A981
:106DB000194801F0EBF8012240F22551164801F084
:106DC00047F90121144801F039F91448056007B06A
:106DD00030BD10B540F225510F4801F05DF9012892
:106DE00009D10E48006830B10B4801F051F9044652
:106DF0000A490968884710BDCC070020E802002036
:106E000000000240EC020020000801400038014070
:106E1000CC060020E402002000440040F0020020E4
:106E200070476D490988490009B201806A4949885B
:106E3000490009B2418068498988490009B28180C6
:106E40007047704770476449C98809B20180624938
:106E5000098909B241806049498909B28180704736
:106E60005E4A02605E4A42605E4A82605B4A0A6035
:106E70005D4A4A605D4A8A604FF4BC725C4B1A807E
:106E8000704770B505460C4615E00520FFF76AFD12
:106E9000284600F0C0FB00BF284600F0C1FB0028D8
:106EA000FAD1284600F0C3FB00BF284600F0C4FB1F
:106EB0000028FAD1641E002CE7DC70BD00B591B04B
:106EC0004C4800F009FC4C480190434802900020D7
:106ED0000390092004900020059080200690400037
:106EE0000790800008902020099000020A9000205E
:106EF0000B9001A93F4800F05CFC01213D4800F0E7
:106F000075FC00200C9001208DF834008DF83500C0
:106F10004FF460200E9000200F9009208DF8400063
:106F20000CA935484C3800F043FB032301220A2109
:106F300031484C3800F091FB032302220B212E48EC
:106F40004C3800F08AFB03231A460C212A484C389F
:106F500000F083FB032304220D2127484C3800F066
:106F60007CFB032305220E2123484C3800F075FBDF
:106F7000032306220F2120484C3800F06EFB032328
:106F8000072205211C484C3800F067FB0323082228
:106F9000062119484C3800F060FB03230922072121
:106FA00015484C3800F059FB012113484C3800F0CB
:106FB00028FB012110484C3800F019FB02210E4833
:106FC0004C38FFF75EFF01210B484C3800F03BFBCB
:106FD00011B000BD00207047CC080020436E0008AF
:106FE000476E0008456E0008236E0008216E0008F9
:106FF000FA010020080002404C2401402DE9FC4128
:107000000646002700256BE0FB4800EBC50103C9DD
:10701000CDE90001F94800EBC5040098B0425DD10C
:10702000BDF80610304600F0A2FF012856D1BDF889
:107030000610009800F0A6FF15B90120F04908706D
:10704000BDF8040030B1042809D008280CD00C2861
:1070500014D10EE0009800F081FF07460EE0009882
:1070600000F07EFF074609E0009800F07BFF07462E
:1070700004E0009800F078FF074600BF00BF2078CA
:1070800008B9678000E0A780207858B901202070F7
:107090000220DC494880BDF804000880009800F018
:1070A00085FE1BE0A0886188884204DDA088618895
:1070B000401AE08006E060884FF6FF71081AA18848
:1070C0000844E08000202070CF490880CD494880E6
:1070D000BDF804000880009800F068FE681CC5B286
:1070E000082D91DBBDE8FC8170B5054602212846DC
:1070F00000F03DFF01280BD1C4480088C449088036
:10710000284600F02BFFC14908800120BC490870C7
:107110000221284600F036FFBC480088BC49098897
:10712000884206DDB9480088B9490988401A84B206
:1071300008E0B74800884FF6FF71081AB34909887C
:10714000084484B2B4F57A6F03DD0020B1490870B9
:1071500019E040F2EE2084420DDD40F6CA00844280
:1071600009DAAC480078082805DAA448A949097862
:1071700000EBC100C480A7480078401CA5490870F6
:107180000020A149088070BD10B5A348007820B147
:107190004FF08040FFF7A8FF03E04FF08040FFF77B
:1071A0002DFF10BD30B585B005460020049001903C
:1071B000029003900090002D46D00120ADF8100001
:1071C00028208DF8130002208DF8120004A993489E
:1071D00000F084FF1C208DF8000000208DF80100D5
:1071E00001208DF802008DF80300684600F0ADF92B
:1071F00001A800F073FE4720ADF804004FF6FF70C1
:10720000ADF808000020ADF8060001A94FF080405D
:1072100000F044FC00207B49488001208880002049
:10722000C880088108804FF0804000F0BFFD012237
:107230000221480700F070FE0121880700F057FE88
:107240000A207749087052E01F20ADF8100028206E
:107250008DF8130002208DF8120004A96F4800F089
:107260003DFF1C208DF8000000208DF8010001205A
:107270008DF802008DF80300684600F066F901A859
:1072800000F02CFE4720ADF804004FF6FF70ADF87B
:1072900008000020ADF8060001A94FF0804000F082
:1072A000FDFB002057494880012088800020C880CD
:1072B000088100240DE0504800EBC400808851494B
:1072C00008804D4951F834004E4900F06FFD601CB4
:1072D000C4B2042CEFDB01221E21900700F01CFE3B
:1072E0000121880700F003FE04204D49087005B015
:1072F00030BD30B589B00446002008900590069056
:1073000007900190029003900490607842490870C1
:10731000002507E040F2DC50384901EBC501C88088
:10732000681CC5B2082DF5DB207818B13A48007802
:10733000FFF738FF4FF47070ADF8200018208DF87B
:10734000230002208DF8220008A9364800F0C6FE6E
:1073500005A800F0C3FD4720ADF81400A08832490D
:1073600091FBF0F0401E80B2ADF8180005A92F483F
:1073700000F094FB7020ADF804000120ADF8060089
:107380000020ADF808004FF47A70ADF80A00022032
:10739000ADF80C00C001ADF8100001A9234800F0C1
:1073A000B6FB01A9214800F0E7FB01A91F4800F046
:1073B0001DFC01A91D4800F051FC08211B4800F0EC
:1073C000B3FD0821194800F0B5FD0821174800F069
:1073D000B8FD0821154800F0BAFD0121134800F05E
:1073E00086FD0121114800F08CFD08210F4800F0B6
:1073F0009BFD002009B030BDF4020020DE08002013
:10740000560300201E0900203801002058030020E8
:107410005A0300205C0300205403002000080140B0
:1074200055030020000C014040420F0000080040BE
:10743000084A1278904203DA074A52F82020118055
:1074400070470146054800EBC100C08870470148FD
:10745000007870475503002034030020DE08002028
:10746000324810B5016841F0010101604168304ABD
:107470001140416001682F4A11400160016821F408
:1074800080210160416821F4FE0141604FF41F0139
:10749000816000F005F828494FF00060086010BDD9
:1074A00022480021026842F4803202604FF4A06357
:1074B000026801F1010112F4003F01D19942F7D1B4
:1074C0000168890330D51D490A6842F010020A603C
:1074D0000A6822F003020A600A6842F002020A60A7
:1074E0004168416041684160416841F480614160A8
:1074F000416821F47C114160416841F4E811416028
:10750000016841F08071016001688901FCD5416822
:1075100021F003014160416841F00201416041688E
:10752000C1F381010229FAD1704700000010024026
:107530000000FFF8FFFFF6FE08ED00E0002002402B
:107540001849084318490860704770B50F21C4787E
:10755000027801234FF0E026DCB1134C246804F4D8
:10756000E064C4F5E064250AC5F10404E940457807
:10757000A54084780C402C4321010C4C1155007817
:1075800000F01F018B40400906EB8000C0F800317D
:1075900070BD02F01F008340500906EB8000C0F868
:1075A000803170BD0000FA050CED00E000E400E061
:1075B00010B54268464B0C791A400B6842EA042227
:1075C000134343608368434A1340D1E90242224394
:1075D0004C7943EA44031A438260C26A097C22F46C
:1075E0007002491EC9B242EA0151C16210BD0029B0
:1075F000816802D041F0010101E021F001018160C8
:1076000070470029816802D041F4807101E021F4C3
:10761000807181607047816841F008018160704726
:10762000014600208968090700D50120704781685C
:1076300041F00401816070470146002089684907D4
:1076400000D5012070470029816802D041F4A001D3
:1076500001E021F4A0018160704770B50725092978
:107660000AD9C468A1F10A0606EB4606B540AC4348
:10767000B3401C43C46007E0046901EB4106B54018
:10768000AC43B3401C4304611F23072A09D2446B57
:10769000521E02EB820293409C4391400C43446390
:1076A00070BD0D2A09D2046BD21F02EB82029340F7
:1076B0009C4391400C43046370BDC46A0D3A02EBD5
:1076C000820293409C4391400C43C46270BD000011
:1076D000FFFEF0FFFDF7F1FF01684FF6FE7211406B
:1076E00001600021016041608160C1604F494F4AE3
:1076F0000839904203D1486840F00F0006E04B4A39
:107700001432904204D1486840F0F000486070475D
:10771000464A2832904203D1486840F47060F5E749
:10772000424A3C32904203D1486840F47040EDE751
:107730003E4A5032904203D1486840F47020E5E759
:107740003A4A6432904203D1486840F47000DDE761
:10775000364A7832904203D1486840F07060D5E7ED
:10776000334A111F904203D1086840F00F0006E031
:107770002F4A1432904204D1086840F0F0000860AB
:1077800070472B4A2832904203D1086840F4706059
:10779000F5E7274A3C32904203D1086840F4704034
:1077A000EDE7234A50329042EAD1086840F4702055
:1077B000E5E730B5036847F6F07293430C6A8A68D0
:1077C0002243D1E904452C4322438C692243CC69EE
:1077D00022434C6A22438C6A22431A430260CA68DD
:1077E00042600A6882604968C16030BD0029016852
:1077F00002D041F0010102E04FF6FE72114001603B
:107800007047002A026801D00A4300E08A43026000
:107810007047406880B27047C10003D50449091F12
:107820000860704701490839486070470800024005
:10783000080402405A4910B588424FF0010101D1B5
:107840004C0501E04FF48004204600F00FF920467B
:10785000BDE81040002100F009B970B504468088E9
:1078600086B00D4620F03F06684600F09FF84D496F
:107870000298B0FBF1F189B20E43A680228822F073
:1078800001022280484B2A689A421CD85200B0FB61
:10789000F2F080B2042800D20420491C2184A08385
:1078A000208840F00100208021884FF6F53001400B
:1078B000A8886A89104308432080A8892989084339
:1078C000208106B070BDEB88A3F53F46FF3E05D191
:1078D00002EB4202B0FBF2F080B208E002EBC2031E
:1078E00003EB0212B0FBF2F080B240F480400205DC
:1078F00001D140F001004FF4967251434FF47A7277
:10790000B1FBF2F140F40040C7E741F28831016079
:10791000002181804BF6FF72C280018141814FF4CA
:107920008041818170470029018802D041F0010126
:1079300001E021F00101018070470029018802D097
:1079400041F4807101E021F48071018070470029C9
:10795000018802D041F4007101E021F4007101803E
:1079600070470029018802D041F4806101E021F4D0
:10797000806101807047002A828801D00A4300E0BC
:107980008A438280704701827047008AC0B2704784
:1079900012B141F0010101E001F0FE0101827047E6
:1079A0000054004040420F00A0860100374910B546
:1079B0004A6812F00C03364A03D0042B01D0082B7E
:1079C00026D002604A68334B02F0F00212099C5C38
:1079D0000268E24042604C6804F4E064240A1C5DE2
:1079E00022FA04F484604C6804F460544FEAD4240E
:1079F0001B5D22FA03F2C2604968264B01F4404144
:107A00004FEA91311B1F595CB2FBF1F1016110BDCE
:107A10004A684B6802F470124FF0020413F4803F7E
:107A200004EB924202D04B689B0301D51A4B00E055
:107A3000174B5A43C5E7154A0029516901D0014344
:107A400000E0814351617047104A0029916901D0DB
:107A5000014300E08143916170470C4A0029D169DC
:107A600001D0014300E08143D1617047074A0029FA
:107A7000116901D0014300E081431161704703485F
:107A8000416A41F08071416270470000001002407D
:107A900000127A007803002000093D0030B502880A
:107AA000F84BF94C98420DD0A0420BD0B0F1804F6A
:107AB00008D0F64DA84205D0F54DA84202D0F54DAC
:107AC000A84203D122F070054A882A43F24DA84209
:107AD00006D0F24DA84203D022F44075CA882A434A
:107AE00002808A8882850A88028598420AD0A0424C
:107AF00008D0EB4A904205D0EA4A904202D0EA4AC6
:107B0000904201D1097A01860121818230BD30B5D0
:107B1000028C22F001020284028C8388048B22F002
:107B2000020224F073050C882C430D8915434A8802
:107B30002A43D44DA8420BD0D34DA84208D0D84DEB
:107B4000A84205D0D74DA84202D0D74DA8420DD1AA
:107B500022F008054A8923F440732A4322F00405E1
:107B60008A882A438D891D43CB892B4383800483D4
:107B7000C9888186028430BD30B5028C22F01002A3
:107B80000284028C8388048B22F0200224F4E645D0
:107B90000C88240645EA14440D892D0542EA154552
:107BA0004A88120545EA1242B64DA84202D0B64DA7
:107BB000A84215D122F080054A8923F440631205BA
:107BC00045EA124222F040058A88120545EA12422F
:107BD0008D89AD0443EA1545CB899B0445EA1343DF
:107BE00083800483C9880187028430BD30B5028C4C
:107BF00022F480720284028C8388848B22F40072C7
:107C000024F073050C882C430D892D0642EA154596
:107C10004A88120645EA12429A4DA84202D09A4D6D
:107C2000A84215D122F400654A8923F44053120674
:107C300045EA124222F480658A88120645EA124219
:107C40008D892D0543EA1545CB891B0545EA13436C
:107C500083808483C9888187028430BD30B5028CDB
:107C600022F480520284038C8288848B24F4E645BB
:107C70000C88240645EA144423F400550B891B079D
:107C800045EA13434D882D0743EA15457D4B98423D
:107C900002D07D4B984205D122F480438A89920517
:107CA00043EA124282808483C988A0F84010058488
:107CB00030BD828B22F440628283828B42EA0122B1
:107CC00082837047828B22F00C028283828B0A436C
:107CD00082837047028B22F440620283028B42EA65
:107CE00001220283704770B5048C24F010040484D0
:107CF000068B048C26F473461B0746EA13431206D0
:107D000043EA12420D055F4B2D0C98420ED05E4B9C
:107D100098420BD0B0F1804F08D05C4B984205D010
:107D20005B4B984202D05B4B984205D124F0200176
:107D3000294341F0100104E024F0A0030B4343F079
:107D400010010283018470BD028B22F00C020283B9
:107D5000028B0A430283704730B5048C24F001047F
:107D60000484058B048C1B0542EA134325F0F305BC
:107D7000444A2B4390420ED0434A90420BD0B0F17C
:107D8000804F08D0414A904205D0414A904202D0EB
:107D9000404A904202D124F0020201E024F00A029B
:107DA0000A4342F001010383018430BD2DE9F05FF5
:107DB0000D4604460E883348DFF8CCC0DFF8CCA06F
:107DC000DFF8CCE04988AA882B894FF0804B3EB37E
:107DD000042E2DD0082E268C32D026F480562684F0
:107DE000B4F81C90268C0F074FEA1748120629F4A6
:107DF00073471B0747EA124242EA134384420AD000
:107E0000644508D05C4506D0544504D0744502D082
:107E10002048844256D126F4005040EA080054E03D
:107E20002046FFF799FFE9882046BDE8F05F8BE721
:107E30002046FFF758FFE9882046BDE8F05F49E794
:107E400026F480762684A78B268C1B0527F0F30763
:107E500042EA13434FEA01683B434FEA1848844221
:107E60000AD0644508D05C4506D0544504D074451A
:107E700002D00848844219D126F4007040EA080074
:107E800017E00000002C01400034014000040040D5
:107E900000080040000C00400010004000140040AA
:107EA00000400140004401400048014026F42060A9
:107EB000084340F48070A3832084E9882046BDE80D
:107EC000F05FFFE626F40240084340F48050A383AD
:107ED0002084E9882046BDE8F05FEAE64FF6FF71AE
:107EE000818000210180C18041800172704700299A
:107EF000018802D041F0010101E021F0010101807F
:107F00007047002930F8441F02D041F4004101E0DD
:107F1000C1F30E0101807047002A828901D00A4313
:107F200000E08A4382817047028B22F008020A43F4
:107F300002837047028B22F4006242EA012101832E
:107F40007047828B22F008020A4382837047828B3B
:107F500022F4006242EA012181837047808E7047DB
:107F6000008F7047808F7047B0F840007047038AD9
:107F7000002280890B4200EA010001D000B10122F9
:107F800010467047C94301827047000030B504466F
:107F9000008A85B00D464CF6FF710840E988014320
:107FA0002182A1894EF6F3100140A8882A89104346
:107FB0006A890A431043A081A08A4FF6FF41084016
:107FC000A9890143A1826846FFF7F0FC4248844238
:107FD00001D1039800E00298A1890904002900EB6F
:107FE000C00101EB0010296802DA4FEA410101E00B
:107FF0004FEA8101B0FBF1F06422B0FBF2F14FEAED
:1080000001114FEA11136FF018056B4300EB830069
:10801000A3891D044FF0320306D503EBC000B0FB6B
:10802000F2F000F0070005E003EB0010B0FBF2F007
:1080300000F00F000843208105B030BD0029818980
:1080400002D041F4005101E021F4005181817047D8
:1080500010B5C1F3421301F01F040121A140012B0F
:1080600007D0022B07D01430002A026805D00A433B
:1080700004E00C30F8E71030F6E78A43026010BDE8
:10808000002A828A01D00A4300E08A438282704734
:108090008088C0F30800704770B501F01F06012208
:1080A0000025C1F3421302FA06F4012B0FD0022B74
:1080B0000FD0838A4FEA11210088234202FA01F28D
:1080C00000EA020001D000B10125284670BD838975
:1080D000F0E7038AEEE70000003801402DE9F041A7
:1080E000CB78002503F00F02DB0601D58B781A430D
:1080F0000B884FF00F0813F0FF0F4FF0010C1CD04E
:10810000D0F800400E880CFA05F31E409E4210D1B4
:10811000AF0008FA07F624EA060602FA07F4344329
:10812000CE78282E02D0482E02D002E0436100E033
:1081300003616D1C082DE5D304600B88FF2B1DD94E
:108140004468002505F108060CFA06F30E881E4067
:108150009E420FD1AF0008FA07F624EA060602FA9B
:1081600007F43443CE78282E00D14361CE78482ED0
:1081700000D103616D1C082DE4D34460BDE8F0819B
:108180000246002092680A4200D001207047016137
:10819000704741617047F0B51C4C002801DAE36973
:1081A00000E06368420D120185B2C0F301579540AB
:1081B000C0F30346032F05D0C2020AD50322B24002
:1081C000934307E023F07062636823F07063636099
:1081D00002E0AB4343F0706201B12A43002801DAA8
:1081E000E261F0BD6260F0BD10B58A0721F00304C2
:1081F0000649130F21440F228C689A4094438C60E7
:108200008A68984002438A6010BD00000000014067
:108210003748364941603749416070473448016901
:1082200041F080010161704731490420CA68D207DA
:1082300001D001207047CA68520701D5022070475B
:10824000C968C906FBD50320704700B50346FFF790
:10825000EBFF02E0FFF7E8FF5B1E012803D0002BD5
:1082600000D1052000BD002BF4D1FAE770B505461A
:108270004FF430263046FFF7E8FF042811D11C4C9C
:10828000206940F0020020616561206940F04000F3
:1082900020613046FFF7D9FF216941F6FD72114098
:1082A000216170BDF0B505464FF4005C0E46604696
:1082B000FFF7CBFF042814D10D4C206940F00100DA
:1082C00020612E806046FFF7C0FF41F6FE7704284C
:1082D00004D1300C68806046FFF7B7FF2169394050
:1082E0002161F0BD0249C860704700002301674565
:1082F00000200240AB89EFCD1848194902680060A0
:108300008A4203D01748804717480047174E4FF05E
:10831000150030601648016821F07061016041026B
:108320000160144C5FF4004020601349134808605A
:10833000134C5FF4805020601249134808601348C2
:10834000D0F800D040680047FEE7FEE7FEE7FEE712
:10835000FEE7FEE7FEE7FEE7FEE7FEE7F04F002060
:10836000EFBEADDE61740008ED0000081810024099
:10837000040001401408014004080140444444340E
:1083800014100140041001404444434400F0FF1F16
:108390000048704738980008A0F16101192900D8F9
:1083A000203870472DE9F05F83460F461546994601
:1083B0004FF0FF36DDF828A011E0A819441009FBA2
:1083C000047080460146584652469047002802D025
:1083D00004DA254603E04046BDE8F09F2646A5EBBB
:1083E00006000128E9DC0020F6E740EA01039B07CC
:1083F00003D009E008C9121F08C0042AFAD203E01A
:1084000011F8013B00F8013B521EF9D27047D2B27D
:1084100001E000F8012B491EFBD270470022F6E76D
:1084200010B504460846114602462046FFF7EFFF06
:10843000204610BD30B50EE003460A4601E05B1C45
:10844000521C1C781578AC4201D1002CF7D115F0E4
:10845000FF0F04D0401C0278002AEDD1002030BD6F
:10846000CAB20178914203D009B1401CF9E700205B
:1084700070470146002000E0401C0A5C002AFBD146
:1084800070472DE9F041054600200E46904604460F
:1084900000E0641C44450BD2285D00F035F9074626
:1084A000305D00F031F9381A02D1295D0029F0D190
:1084B000BDE8F08170B5064600F0A4FA04680546F0
:1084C0000A220021304600F025F92C6070BDF0B47E
:1084D00080EA0102D20F4300B3EB410F02D2034600
:1084E000084619464B0042D0C30DDDB2C1F3C75454
:1084F0002C1B202C35DAC1F3160141F4000502B122
:108500006D42C4F1200605FA06F125412844B3EB7B
:10851000D05F23D0C2B1012CA0EBC35009DCF0BC6A
:108520004FF0004202EAC35200F50000DBB200F057
:1085300032B9400000F1807000EBC350A0F18070B0
:1085400040EAD170490009E0490841EAC071A0EB56
:10855000C35000F50000400800EBC350F0BC00F031
:1085600011B95142012303EB4101801AF6E7F0BC37
:10857000704781F00041AAE780F00040A7E780EA59
:10858000010210B502F00042400026D04B0023D07B
:108590004FEA106101EB1361C0F35600C3F35603B9
:1085A00040F4000043F40003A0FB0330A1F17F017D
:1085B0004FEA00401C0401D000F1010050EA1340D2
:1085C00001D44000491EC3B20C0604EBD010401C7D
:1085D0004008802B02D003E0002010BD20F00100F5
:1085E000002900DA0020104310BD80EA010202F0E9
:1085F000004330B430F0004221F0004015D0A0B16B
:10860000C0F3C755C2F3C754C2F31601C0F3160036
:10861000651B41F4000140F400007D35814201D327
:108620006D1C00E04900002D02DA30BC00207047CC
:108630004FF400020024814201D3091A1443520866
:108640004FEA4101F7D151B1814202D14FF00041CF
:1086500005E002D24FF0010101E06FF0010104EBEF
:10866000C55030BC184400F08DB8C10F80EAE070EE
:108670000844CA079623002100F08DB896230022F3
:10868000114600F088B800F0004220F00040C10D13
:10869000C0F3160040F400007F2901DA0020704783
:1086A000962903DCC1F19601C84001E09639884063
:1086B000002AF4D04042704720F00040C10DC0F3C2
:1086C000160040F400007F2901DA00207047962947
:1086D00003DCC1F19601C840704796398840704765
:1086E000002801DBC0F10040002901DBC1F100419D
:1086F00081427047002801DBC0F10040002901DB06
:10870000C1F1004188427047A0F14101192900D808
:10871000203070472DE9F0470F46914680460446C9
:10872000002614F8015B2DB1FFF732FE0068405DB2
:10873000C007F6D12B2D02D02D2D18D0641E4A462D
:108740003946204600F0C0F827B13968A14201D16E
:10875000C7F8008071054FF002040BD54042002895
:1087600003DD00F04FF90460A007BDE8F08746F490
:108770008066E4E70028F8DA00F044F904606FF05E
:108780000040F2E70029A8BF7047401C490008BF1D
:1087900020F00100704710B4B0FA80FC00FA0CF031
:1087A00050EA010404BF10BC704749B1CCF1200469
:1087B00021FA04F411FA0CF118BF012121430843F6
:1087C000A3EB0C01CB1D0106000A002BBEBF00204D
:1087D00010BC704700EBC35010440029A4BF10BC6C
:1087E0007047401C490008BF20F0010010BC7047D2
:1087F000420005D0C0F3C7525242914201DC002032
:10880000704700EBC1507047F0B4002802DCF0BCA8
:1088100000207047C0F3C751C0F3160040F40000B9
:10882000CA0701D14000491E3F2202EB6105002228
:1088300011464FF4000626FA01F31344D41884427B
:1088400001D8001B1A464000491C1729F3DD5100CE
:10885000814202D24FF0FF3100E0002102EBC5500F
:10886000F0BCFFF78FBF10B541000CD0C0F3C7516B
:10887000962908DC7E2909DC06DB410204D000F0E1
:10888000004040F07E5010BD002010BDC1F19604A4
:10889000C4F1200100FA01F1E040FFF773FFA040AE
:1088A00010BD0000064C074D06E0E06840F00103F3
:1088B00094E8070098471034AC42F6D3F7F71AFC57
:1088C000889D0008A89D00082DE9F05F8246007889
:1088D00000278B4615460AF10104B946302801D01D
:1088E0009DB113E014F8010B0127782803D0582814
:1088F00001D045B10AE00DB1102D07D10027102598
:1089000014F8010B02E0082500E00A250026B04615
:108910000EE005FB080005FB06F1012701EB104600
:108920001FFA80F8B6F5803F00D3B94614F8010B62
:10893000294600F018F80028EBDABBF1000F05D04B
:108940000FB1641E00E05446CBF80040B9F1000FAF
:1089500006D000F057F802210160C81EBDE8F09F64
:1089600048EA0640FAE73A2800D2303820F02002E0
:10897000412A01D3A2F13700884201D34FF0FF30E2
:10898000704770B501EB020410F8015B15F00703A6
:1089900001D110F8013B2A1106D110F8012B03E098
:1089A00010F8016B01F8016B5B1EF9D12B0705D4A0
:1089B0000023521E0FD401F8013BFAE710F8013BE7
:1089C00002F10202A1EB030303E013F8015B01F8DB
:1089D000015B521EF9D5A142D6D3002070BD4100E3
:1089E000080218BF04200A0E18BF40F001004FF023
:1089F0007F4232EA010108BF40F00200012808BFAF
:108A00000520704700487047880300206FF05E0122
:108A10000807FFF7EDBE00002DE9F04D03461446B0
:108A20004FF07F400E46B0EB440F04D800160860AC
:108A30001846BDE8F08D4FF0004040EA0421C4F331
:108A4000C7507838431100F01F00DFF814C1C0F19F
:108A50002002FC445CF823500CEB83038540D3F8E0
:108A600004C02CFA02F72F439D680CFA00FC25FA8B
:108A700002F8DB6805FA00F023FA02F240EA020588
:108A80004CEA080CA7FB0123ACFB01C0A5FB01517C
:108A900001EB0C05A94294BF4FF0000C4FF0010C04
:108AA00081186144BCF1000F02D0814202D903E079
:108AB000814201D2012000E00020184400F1200290
:108AC0004FEA92188006CA0C40EA42304F03C6F8BB
:108AD0000080FFF7CAFD82463846FFF7CFFD6FF0F2
:108AE0001201FFF785FE07462846FFF7C7FD6FF026
:108AF0002501FFF77DFE834639465046FFF7E7FC28
:108B00005946FFF7E4FC00F500656FF30B0551468D
:108B10002846FFF72EFD3946FFF72BFD5946FFF794
:108B20002BFD1049FFF72BFD07460F492846FFF79D
:108B300026FD3946FFF7CBFC07460C492846FFF7D0
:108B40001EFD3946FFF7C3FC14F0004F08BFBDE817
:108B5000F08DC8F1805180F000403160BDE8F08DAB
:108B6000E60D0000DB0FC92F22AAFD290000C92F46
:108B700002E008C8121F08C1002AFAD170477047E6
:108B8000002001E001C1121F002AFBD17047000044
:108B90000149086070470000880300202DE9F04774
:108BA0004FF0684202EB400305460C46B3F1654FB7
:108BB0003CBF02EB4102B2F1654F3FD34FF07F4221
:108BC000B2EB400F28BFB2EB410F03D2BDE8F04734
:108BD000FFF77DBC40EA01035B0008BF44F0FF41A2
:108BE0000AD0B2EB400F08BFB2EB410F06D125F01F
:108BF000804024F0804105460C461FE0B2EB400F58
:108C000012BF5FEA410245F0FF4004F0004115D079
:108C10004FEA410292EA400310D4002AACBF4FF061
:108C20009F464FF03E563146FFF7A9FC05463146B8
:108C30002046FFF7A4FC044628462146C0F3C7524D
:108C4000C1F3C753D21A1B2A06DD10F0004F14BF20
:108C500054485548BDE8F08712F11A0F17DA11F0A1
:108C6000004F06D010F0004F14BF50485048BDE8E8
:108C7000F08721462846FFF7B8FC0446FFF7AFFE11
:108C8000042808BFFFF7C2FE2046BDE8F087420077
:108C9000B2EB410F25D910F0004F19BF454F464E9A
:108CA000464F474E224685F0004415460A4680F05E
:108CB000004110460A1A5200B2F1807F3ED248406D
:108CC0004049DFF804A110F0004F18D04FF03F48A2
:108CD0003846FFF74EFC074651463046FFF749FC41
:108CE00017E011F0004F04BF00263746E2D010F025
:108CF000004F19BF354F364E364F374EDAE74FF03B
:108D00007C583846FFF7E3FB074651463046FFF7ED
:108D1000DEFB064641462846FFF731FC2146FFF7B9
:108D2000D6FB824621464046FFF729FC2946FFF73D
:108D300023FC5146FFF759FC044604E0214628462F
:108D4000FFF753FC04460146FFF719FC8046234910
:108D5000FFF715FC2249FFF7BAFB4146FFF70FFC6E
:108D60002049FFF7B4FB4146FFF709FC1E49FFF716
:108D7000AEFB4146FFF703FC1C49FFF7A8FB054685
:108D800041462046FFF7FBFB2946FFF7F8FB31463B
:108D9000FFF79DFB2146FFF79AFB3946BDE8F047F8
:108DA000FFF795BBDB0FC9BFDB0FC93FDB0F49C026
:108DB000DB0F49400000C9BF22AAFDB90000C93F2E
:108DC00022AAFD390060ED3EC30ACE37000049C03B
:108DD00022AA7DBA0000494022AA7D3A2DAD65BD88
:108DE0008FB8D53D0FB511BE61C84C3EA8AAAABE2A
:108DF0002DE9F8430446024650486946B0EB420F5D
:108E000009D94FF0E640B0EB420F8CBF4FF0FF3076
:108E10000020009034E04A4B22F0004083422BD9DE
:108E200048492046FFF7ABFBFFF71DFD0546FFF75E
:108E30002AFC00F00300009043492846FFF79FFBFF
:108E4000064642492846FFF79AFB0746404928460E
:108E5000FFF795FB80463F492846FFF790FB2146E8
:108E6000FFF78AFB4146FFF784FB3946FFF781FB9A
:108E70003146FFF77EFB02E01046FFF7CDFD0446CA
:108E8000009D002D18DA6000B0F17F4F3CBF4FF01D
:108E90007E50BDE8F88309D14FF00100FFF778FE5E
:108EA000BDE8F84300210846FFF79FBB2046BDE818
:108EB000F8430121FFF79CBC214615F0010F08463D
:108EC0001DD0FFF75CFB06462349FFF758FB2349FB
:108ED000FFF752FB3146FFF752FB2149FFF7F7FA44
:108EE0003146FFF74CFB2146FFF749FB2146FFF7D0
:108EF000EEFA15F0020F18BFBDE8F8831AE0FFF78D
:108F00003EFB04461749FFF73AFB1749FFF7DFFA24
:108F10002146FFF734FB1549FFF7D9FA2146FFF741
:108F20002EFB4FF07E51FFF7D2FA15F0020F08BF6B
:108F3000BDE8F88380F00040BDE8F883B61F927E5C
:108F4000490E494683F9223F1A61342C0020A2338E
:108F500000A0FD390000C93F336D4C39DA82083C6E
:108F6000A0AA2ABEB93AB2BACA9F2A3DDDFFFFBE07
:108F70002DE9F8430446544822466946B0EB420FB7
:108F800009D94FF0E640B0EB440F8CBF4FF0FF30F3
:108F90000020009034E04D4B22F0004083422BD95A
:108FA0004B491046FFF7EBFAFFF75DFC0646FFF76B
:108FB0006AFB00F00300009046493046FFF7DFFAF5
:108FC000054645493046FFF7DAFA07464349304639
:108FD000FFF7D5FA804642493046FFF7D0FA2146DE
:108FE000FFF7CAFA4146FFF7C4FA3946FFF7C1FA5C
:108FF0002946FFF7BEFA02E01046FFF70DFD0446D2
:10900000009D002D1DDA6000B0F17F4F09D220468F
:10901000FFF7E5FC042808BFFFF7F8FC2046BDE891
:10902000F88308D10120FFF7B3FDBDE8F843002124
:109030000846FFF7DABA2046BDE8F8430121FFF7FA
:10904000D7BB214615F0010F08461FD0FFF797FA4E
:1090500004462449FFF793FA2349FFF738FA2146DB
:10906000FFF78DFA2149FFF732FA2146FFF787FA19
:109070004FF07E51FFF72BFA15F0020F08BFBDE845
:10908000F88300BF80F00040BDE8F883FFF777FA6F
:1090900006461749FFF773FA1649FFF76DFA31468E
:1090A000FFF76DFA1449FFF712FA3146FFF767FA36
:1090B0002146FFF764FA2146FFF709FA15F0020F7F
:1090C000E0D1BDE8F8830000B61F927E490E494604
:1090D00083F9223F1A61342C0020A23300A0FD390D
:1090E0000000C93FB93AB2BACA9F2A3DDDFFFFBEB0
:1090F000336D4C39DA82083CA0AA2ABE70B5054609
:10910000FFF782FB044620F00040C0F1FF40C00F93
:1091100008D025F00040C0F1FF40C00F04BF01207F
:10912000FFF736FD204670BD6E9C0008C39C00080A
:10913000990100089C9C0008869D0008E101000838
:109140003F9A0008169B0008050200080B9C0008C7
:10915000869D000811030008079C0008109C000869
:109160005D0300082C9C0008E09C0008E103000857
:10917000909A0008B39C0008BD010008989C000864
:10918000F39C0008FD060008919C0008859C0008DF
:1091900015080008C29B0008869D00080F090008FA
:1091A000AC990008000000001F040020000000002F
:1091B00020000000A9990008000000002004002001
:1091C0000000000064000000FC9A0008000000009D
:1091D0002104002001000000FA000000639900084B
:1091E0000200000024040020B0040000A4060000D7
:1091F000119A000802000000300400200000000066
:10920000D00700001D9A0008020000003204002070
:1092100000000000D0070000B5990008020000001F
:109220003404002000000000D0070000EA9A000883
:10923000020000002604002000000000D00700000B
:10924000F39A00080200000028040020000000003B
:10925000D0070000579B0008000000002A040020EF
:109260000000000001000000659D000800000000F3
:109270002B04002000000000C8000000749D0008BE
:10928000000000002C04002000000000C8000000C6
:10929000FF990008020000002E040020E8030000EF
:1092A000D0070000569A0008020000003604002093
:1092B00032000000F2010000479A0008020000009E
:1092C0003804002032000000F2010000739A000808
:1092D0000400000064040020B004000000C201008B
:1092E000839A00080400000054040020B004000029
:1092F00000C20100529C000800000000220400206F
:109300000000000001000000E699000800000000D5
:10931000140400200A000000C8000000D3990008CF
:1093200000000000150400200A00000032000000C8
:10933000C099000800000000160400200A00000088
:1093400032000000DA9B0008010000003A0400200F
:10935000FFFFFFFF01000000F0990008020000007D
:109360003C04002000000000D0070000B69B00086D
:10937000020000003E04002000000000D0070000B2
:10938000599D000802000000400400200000000079
:10939000D0070000619C0008000000004404002089
:1093A00000000000FF000000649B000801000000B6
:1093B000420400209CFFFFFF64000000769B000831
:1093C00001000000430400209CFFFFFF6400000038
:1093D000959B000802000000460400206400000085
:1093E000B80B0000389D000802000000480400206F
:1093F00064000000B80B000088990008020000001B
:109400004A04002064000000B80B0000A69B00087E
:10941000020000004C04002064000000B80B0000B3
:10942000499D0008020000004E0400206400000076
:10943000B80B0000999900080200000050040020B9
:1094400064000000B80B0000329A00080000000021
:10945000EE0300200000000003000000329C000822
:1094600000000000EF03002000000000FA000000F0
:10947000959A000802000000F003002000000000A0
:1094800000010000419C000802000000F2030020DF
:1094900064000000E8030000CA9B0008030000000D
:1094A000E8030020B0B9FFFF50460000F39B00081E
:1094B00000000000BA03002000000000C800000007
:1094C000D69A000800000000C4030020000000003D
:1094D000C80000007499000800000000CE030020BE
:1094E00000000000C8000000E89B00080000000029
:1094F000BB03002000000000C8000000CB9A000859
:1095000000000000C503002000000000C8000000AB
:109510006999000800000000CF030020000000004F
:10952000C8000000FD9B000800000000BC030020F4
:1095300000000000C8000000E09A000800000000E1
:10954000C603002000000000C80000007E9900084B
:1095500000000000D003002000000000C800000050
:10956000779C000802000000580400200000000062
:10957000D00700009E9A0008000000005C04002054
:109580000000000001000000879B000802000000AE
:109590005E0400200A000000D00700002A9D000899
:1095A00002000000600400200A000000D007000054
:1095B000659A0008000000005B0400200000000025
:1095C00064000000299A000802000000B403002093
:1095D000DC05000028230000C39A000800000000FA
:1095E000B703002000000000C8000000BB9A00087C
:1095F00000000000C103002000000000C8000000BF
:10960000B39A000800000000CB0300200000000017
:10961000C8000000509B000800000000B6030020B6
:1096200000000000C8000000499B00080000000086
:10963000C003002000000000C8000000429B00089A
:1096400000000000CA03002000000000C800000065
:109650001C9D000800000000B8030020000000006E
:10966000C8000000169D000800000000C203002092
:1096700000000000C8000000109D0008000000006D
:10968000CC03002000000000C8000000AD9C0008D2
:1096900000000000B903002000000000C800000026
:1096A000A79C000800000000C30300200000000089
:1096B000C8000000A19C000800000000CD030020AD
:1096C00000000000C80000003A9B000800000000F5
:1096D000BD03002000000000C8000000329B00080D
:1096E00000000000C703002000000000C8000000C8
:1096F0002A9B000800000000D103002000000000A9
:10970000C8000000414552543132333400414343D4
:109710003B4241524F3B4D41473B43414D535441E6
:10972000423B43414D545249473B41524D3B4750C8
:109730005320484F4D453B47505320484F4C443BE6
:1097400050415353544852553B4845414446524575
:10975000453B4245455045523B4C45444D41583BA5
:109760004C4C49474854533B4845414441444A3B8B
:1097700000524F4C4C3B50495443483B5941573B96
:10978000414C543B506F733B506F73523B4E61766C
:10979000523B4C4556454C3B4D41473B56454C3B57
:1097A00000000000001001400010100000080140FF
:1097B0000080100000404040404040404040414157
:1097C0004141414040404040404040404040404096
:1097D0004040404040050202020202020202020230
:1097E000020202020220202020202020202020022D
:1097F00002020202020290909090909010101010BD
:109800001010101010101010101010101010101058
:1098100002020202020288888888888808080808EC
:1098200008080808080808080808080808080808B8
:109830000202020240000000B5970008000000008C
:109840006E83F9A22915444ED15727FCC0DD34F5AB
:10985000999562DB4190433CAB6351FE4D505536C8
:1098600030353000565441494C340059340041449D
:10987000584C3334350048455836005936004F436C
:10988000544F583800414343004641494C534146E8
:109890004500414952504C414E45004D414700481A
:1098A000454C495F39305F444547004759524F5F47
:1098B000534D4F4F5448494E47004C45445F524921
:1098C0004E4700464C59494E475F57494E47004264
:1098D00049005452490047494D42414C00494E46C7
:1098E0004C494748545F4143435F43414C0048451E
:1098F0004C495F3132305F4343504D0050504D0072
:109900005350454B5452554D004241524F00515512
:10991000414450004D4F544F525F53544F50004FED
:1099200043544F464C41545000534F4E4152004710
:109930005053005642415400534552564F5F5449CC
:109940004C54004845583658005155414458004F32
:1099500043544F464C4154580054454C454D455492
:109960005259006D69647263006770735F706F7342
:10997000725F64006770735F706F735F640067701D
:10998000735F6E61765F640067696D62616C5F70C2
:10999000697463685F6D69640067696D62616C5FBB
:1099A000726F6C6C5F6D6964007961776465616486
:1099B00062616E64006D696E636F6D6D616E6400EF
:1099C000766261746D696E63656C6C766F6C7461E0
:1099D000676500766261746D617863656C6C766F43
:1099E0006C7461676500766261747363616C6500B5
:1099F0007472695F7961775F6D6964646C65006634
:109A000061696C736166655F7468726F74746C65AC
:109A1000006D696E7468726F74746C65006D617846
:109A20007468726F74746C65006C6F6F7074696DBC
:109A300065006163635F6861726477617265006687
:109A400065617475726500736572766F5F70776DAE
:109A50005F72617465006D6F746F725F70776D5FB8
:109A600072617465006E61765F736C65775F7261B9
:109A700074650073657269616C5F626175647261BF
:109A80007465006770735F6261756472617465000C
:109A900073617665006779726F5F6C7066006E61E6
:109AA000765F636F6E74726F6C735F686561646913
:109AB0006E6700645F706974636800695F706974E1
:109AC000636800705F7069746368006770735F70CB
:109AD0006F73725F69006770735F706F735F6900A7
:109AE0006770735F6E61765F69006D696E6368654C
:109AF000636B006D6178636865636B00616C745FB4
:109B0000686F6C645F7468726F74746C655F6E65A7
:109B1000757472616C006C697374206F72202D769D
:109B2000616C206F722076616C00645F6C65766595
:109B30006C00695F6C6576656C00705F6C6576655E
:109B40006C00645F726F6C6C00695F726F6C6C00AC
:109B5000705F726F6C6C0072657461726465645FD3
:109B600061726D0067696D62616C5F7069746368D2
:109B70005F6761696E0067696D62616C5F726F6CCF
:109B80006C5F6761696E006E61765F7370656564B6
:109B90005F6D696E0067696D62616C5F70697463A7
:109BA000685F6D696E0067696D62616C5F726F6C92
:109BB0006C5F6D696E007472695F7961775F6D6962
:109BC0006E0076657273696F6E006D61675F6465C4
:109BD000636C696E6174696F6E007961775F646947
:109BE00072656374696F6E006770735F706F737214
:109BF0005F70006770735F706F735F700067707382
:109C00005F6E61765F70006D61700068656C7000FA
:109C10006D617070696E67206F6620726320636883
:109C2000616E6E656C206F72646572006D69786537
:109C300072006163635F6C70665F666163746F720C
:109C4000006779726F5F636D70665F666163746FE2
:109C500072007370656B7472756D5F68697265739D
:109C60000067696D62616C5F666C61677300646553
:109C70006661756C7473006770735F77705F726193
:109C8000646975730073686F772073797374656D99
:109C900020737461747573007365740065786974FA
:109CA00000645F616C7400695F616C7400705F6177
:109CB0006C74007361766520616E64207265626FFA
:109CC0006F7400726573657420746F2064656661DB
:109CD000756C747320616E64207265626F6F7400BE
:109CE0006D69786572206E616D65206F72206C6998
:109CF0007374006E616D653D76616C7565206F7281
:109D000020626C616E6B20666F72206C69737400E8
:109D1000645F79617700695F79617700705F79616D
:109D200077004D4D4138343578006E61765F737041
:109D30006565645F6D61780067696D62616C5F7015
:109D4000697463685F6D61780067696D62616C5FFB
:109D5000726F6C6C5F6D6178007472695F796177A6
:109D60005F6D6178006661696C736166655F6465EB
:109D70006C6179006661696C736166655F6F6666C8
:109D80005F64656C61790000A89D000800000020F8
:109D90008C03000082890008889E00088C03002044
:109DA0009C150000808B00084113D29814080E996E
:109DB0001B0849041ACF0C1AD6041A7B041A76041D
:109DC0001AC3041A6B041A431C1A7E081A1F081AB5
:109DD0004F041A920C1AEE041A9F041A6404411AD2
:109DE000FC081A331C2ADD1019081A14041A380446
:109DF0001AAB101ABA041A2F0C1A89081A29081A51
:109E00005904411A85101A090C5A9B182924411328
:109E1000869D1B086E141A5C041A220C81026318BA
:109E20001204CBDC05020116092426210296030246
:109E3000FB0122403A020812043A040812083A08C8
:109E400008120C22105A0420190839201908392048
:109E5000190829201334081B4038041A3C04191926
:109E60001B4034181A38041A3C041931193CB13B10
:109E7000A24A6141380C01020304060708090204E2
:089E8000066D29106914410070
:04000005080000ED02
:00000001FF
